:020000041000EA
:1000000000B5324B212058609868022188439860DF
:10001000D860186158612E4B002199600221596106
:100020000121F02299502B49196001219960352056
:1000300000F044F80222904214D00621196600F024
:1000400034F8196E01211966002018661A6600F04E
:100050002CF8196E196E196E052000F02FF8012189
:100060000842F9D1002199601B49196000215960AB
:100070001A491B48016001219960EB211966A021F2
:10008000196600F012F800219960164914480160C1
:100090000121996001BC002800D000471248134993
:1000A000086003C880F30888084703B5996A0420EC
:1000B0000142FBD001200142F8D103BD02B5186610
:1000C0001866FFF7F2FF186E186E02BD00000240BE
:1000D000000000180000070000035F00212200005C
:1000E000F4000018222000A00001001008ED00E03C
:1000F00000000000000000000000000074B24E7A12
:1001000000200420F7010010C3010010C5010010F9
:10011000C1010010C1010010C1010010C101001097
:10012000C1010010C1010010C1010010C701001081
:10013000C1010010C1010010C9010010CB01001065
:10014000CD010010CD010010CD010010CD01001037
:10015000CD010010CD010010CD010010CD01001027
:10016000CD010010CD010010CD010010CD01001017
:10017000CD010010CD010010CD010010CD01001007
:10018000CD010010CD010010CD010010CD010010F7
:10019000CD010010CD010010CD010010CD010010E7
:1001A000CD010010CD010010CD010010CD010010D7
:1001B000CD010010CD010010CD010010CD010010C7
:1001C00000BE00BE00BE00BE00BE00BEEFF3058054
:1001D000103800BEF2EB88714465001060650010B5
:1001E0003402001090A31AE700201F49086006C8D7
:1001F00081F3088810471D48006800282FD10DA4FE
:100200000ECC002902D000F012F8F9E71849194A7B
:10021000002000E001C19142FCD1174988471749ED
:1002200088471749884700BEFDE701C901C29A42C5
:10023000FBD3704760650010C00000202408002038
:10024000C46C00100000042000000420C46C0010E6
:10025000001004200010042000000000704709482E
:1002600003F0B6F90047000008ED00E0000000D000
:10027000280800208C0D0020E1220010E10500106C
:10028000A12200105756000006005250ABB3605335
:100290001864001006005250861C030228640010E7
:1002A000060052505422A29D3064001005005250A6
:1002B000DE65F468C46C0010F8B5C0460448054B10
:1002C00010B5834203D0044B002B00D0984710BDDB
:1002D00024080020240800200000000006480749E8
:1002E000091A8B10C90FC91810B5491003D0044B57
:1002F000002B00D0984710BD2408002024080020BF
:100300000000000010B5074C2378002B09D1FFF73F
:10031000D5FF054B002B02D0044800E000BF0123AD
:10032000237010BD2809002000000000E8540010D0
:10033000054B10B5002B03D00449054800E000BF71
:10034000FFF7CCFF10BDC046000000002C090020C4
:10035000E854001070B506000D1C081C04F038F8B5
:1003600084B2002C12D0200004F00AF8011C281CD2
:1003700003F0DDFF8721C90503F0F9FF04F028F839
:10038000C3B21B0224041C43346070BD0023F8E791
:1003900010B504001022002104F0E0F880235B0275
:1003A0002360F8235B0263608023DB02A360C02329
:1003B0001B03A360200010BD70B504000D00FFF703
:1003C000E7FF6A1C636809490B40ED012B431203E8
:1003D00013436360E268D200D208802189050A4392
:1003E000E260034A13406360200070BD7F00FEFF9F
:1003F000FFFFFF9F70B584B006000C0001AB02AA9E
:1004000003A900F0ADFA051E04D1002C09D120008B
:1004100004B070BD019A0299039800F065FA2C00AF
:10042000F5E70248310001F0D7FFC046E85400105C
:10043000F0B5CE46474680B587B004000F00914620
:100440001E00284B98424BD007252900300000F0B1
:10045000DFFA29000E9800F0DBFA0123984600939A
:1004600032003900200004F0CFFA434600930E9A80
:100470003900200004F0C8FA494602A8FFF79CFFA3
:10048000059D194B1D400E9B9B021D430595174B67
:100490001D402E4380235B0333430593049B9B0045
:1004A0009B088022D205134304930F9902A8FFF7FB
:1004B00051FF049A0E4B1A4080239B02134304936E
:1004C00002AB4A463900200004F0F0FA22684346A5
:1004D000BB401343236007B0C0BCB946B046F0BD73
:1004E0000625B2E700002050FF83FFFFE0FF0FFC6E
:1004F000FFFFF5C110B50C2906D80368054A134063
:10050000C9020B43036010BD034B044A0448C321D6
:1005100001F0CAFEFF87FFFF1C550010185600109F
:100520003C55001000B583B0010000230193103347
:100530000193134B019301A8FFF7DCFF019B0C22F1
:10054000190091430A0008210A4301920D4A1A40FA
:100550000A4301920C4A1A400A4301920B4A1A407C
:100560001143019109210A430192094A1A400A43A1
:100570000192084818400843019003B000BDC046EE
:1005800010801F0033F8FFFF33F8BFFF33F89FFFE1
:1005900033F81FFF31F81FFF10B5002B02DB02609C
:1005A000436010BD024B034A03483F2101F07CFE2B
:1005B0009455001000560010B055001010B582B0D0
:1005C000040001F023FA02000B006846FFF7E4FF85
:1005D000009A019B22606360200002B010BD000001
:1005E00030B587B001212348FFF704FF2249234C8F
:1005F000200004F0EDF90200FE239B050193112376
:100600000093013300212000FFF712FF012004F0C6
:10061000A5FA0400FFF786FF194B1840082318437A
:10062000A301A022D2059446634400221A60154A11
:100630005A60802252019A6018611348210000F02C
:10064000E5F802A8FFF7BAFF029C039D002000F026
:1006500019F90E4800F016F9002000F013F902A86D
:10066000FFF7ACFF029A039B121BAB410492059368
:10067000E7E7C046400D0300585600100000205028
:10068000F37FE0FF1000205034560010FFFF000001
:10069000F0B5C64600B590461D00069F780880005C
:1006A00003F046FF0600002200240AE06300595BC5
:1006B0000904631C5B005B5B19439300F150023437
:1006C0000132BC42F2D343469B01A022D20594469C
:1006D0006344DE63642001F01AF9300003F032FF56
:1006E00080BCB846F0BD000070B504000D000120CC
:1006F000002101F0FFF80B49486901231A008240EC
:1007000009698B40134384408D402C43D02212064C
:1007100011694C401C40D4610120002101F0EAF82D
:1007200070BDC046600D0020F0B5D6464F46464627
:10073000C0B505000F00140099460B0018330126C0
:100740009E408660AB683342FCD000210020FFF75A
:10075000CBFF631C9A4621786A683B001033012462
:100760009C402300134098461442F5D10437BF0043
:10077000EF1939704B46012B18D9AE60AB68334284
:10078000FCD000210120FFF7AFFF0BE053460133FF
:10079000524611786A682242FCD13970012294468F
:1007A000E0449A464B46013B4345EFD8AE60AB6808
:1007B0003342FCD001210120FFF796FFE0BCBA468E
:1007C000B146A846F0BD70B506000D0014000AE061
:1007D000A21C29003000FFF7A7FFC82001F097F8FE
:1007E00023780233E4182378002BF1D170BD00B5D3
:1007F00083B06B46DA1D2C2313702B3BFFF794FF5D
:1008000000210120FFF770FF03B000BD70B50D009F
:10081000194C24220100200003F0A6FE174B1D6096
:10082000206900F00DF9606900F00AF9A06900F094
:1008300007F9E06900F004F92369012632009A40C3
:10084000D0252D066A626369310099406962A36907
:10085000310099400B006962E169300088406862AC
:100860006A616B61064A61682068FFF7ACFFE36963
:100870009E406E6170BDC046600D0020240B0020BC
:1008800064560010F0B583B00500154B5968186820
:10089000FFF7ADFF8020800103F04AFE0400002333
:1008A00002E05A00A5520133802252019342F8D34C
:1008B0000C4F3A680A4D69682868802676010096D0
:1008C0002300FFF7E5FE3A68696828680096230070
:1008D000FFF7DEFE200003F035FE03B0F0BDC0469A
:1008E000600D0020240B0020F0B583B004000D0043
:1008F000160000F0B1F8002801D003B0F0BD154F8C
:1009000000973B0001220121053001F0F1FA009629
:100910002B0022000121104801F0F2FB3100694355
:10092000200002F0A9FE04000C4B009300220221DB
:10093000042001F0DDFA00942300002201210520AB
:1009400001F0D6FA00973B0002220021062001F0B8
:10095000CFFAD2E7006CDC0200800240001BB70037
:10096000F0B5DE4657464E464546E0B583B0804674
:100970008B4600920193042001F0BCFBFA21890010
:1009800002F07AFE8246A0235B0099462CE0013CEF
:10099000002C20D025007D432900300002F06CFEA1
:1009A0004045F4D12900300002F066FE0029EED166
:1009B00073019B1B9B009B19DB005A461360009B35
:1009C0001F60019B1C60012003B0F0BCBB46B24617
:1009D000A946A046F0BD013F002F01D03C00D7E75B
:1009E00001235B429C46E1444B460F2B09D95646F6
:1009F0004B465E43044BF218044B9A42F0D807274B
:100A0000EAE70020E0E7C046508EF4FF50F80C0003
:100A100010B58300084A944663441A684024624033
:100A2000803414408022520113431C60C000034BE9
:100A30009C466044416010BD04C00140004001403C
:100A400010B501238340D0221206936293610521E1
:100A5000FFF7DEFF10BD0000034B1B6802201840AB
:100A6000431E9841C0B2704700C00640EFF31080AB
:100A700072B6034B1B68002BFBD0BFF35F8F704730
:100A80002C0100D0BFF35F8F024B00221A6080F36D
:100A9000108870472C0100D0F8B506000C00150036
:100AA000FFF7E4FFE308F718F15C07222240012377
:100AB00093400B4205D1DBB20B433B70FFF7E2FFE3
:100AC000F8BD2100280001F087FCF0B583B00600D6
:100AD000019114001F00FFF7C9FF00E00134BC4280
:100AE0000CD8E308F518F35C0721214001228A4065
:100AF0001A42F3D1D2B21A432A7001E001246442AF
:100B0000FFF7C0FF002C02DB200003B0F0BD019B0B
:100B1000002BF9D0089801F05FFC0000002307E0EB
:100B2000054A9A189200BFF35F8F002111600133CC
:100B30001F2BF5D97047C04640000034054A107895
:100B4000431CDBB21370172B02D9130010221A704A
:100B50007047C04638020020074B9B681030800069
:100B60001950BFF35F8FBFF35F8F044B00211960F3
:100B700082F310887047C04600ED00E0240100D0E9
:100B800010B50388DA0A1C2A05D15B055B15023310
:100B90005B00C01810BD034B034A0448B12101F0AB
:100BA00083FBC046885600102C580010A056001039
:100BB00010B5091A0B1F0A4A88180A4A904208D829
:100BC000C90706D45B105B055B0D0748184380B26C
:100BD00010BD064B064A0748A32101F065FBC0463D
:100BE000FC070000FE0F000000E0FFFFE8560010C9
:100BF00020580010A056001010B5091A04394A08F0
:100C0000090B08D14905490D064B0B430380064BE0
:100C10001343438010BD054B054A0648AB2101F044
:100C200043FBC04600F0FFFF00F8FFFF185700101D
:100C3000F4570010A056001001238340034A1068A7
:100C40001840431E9841C0B27047C04600E100E022
:100C5000002904D0034B1860034B18607047034B06
:100C60001860FBE780E200E000E100E080E100E0E6
:100C700010B5012383401800FFF7EAFF10BD000004
:100C8000024B9B6810308000C058704700ED00E0B8
:100C900070B504000D00EFF3108672B60C4B1B68A4
:100CA000002BFBD0BFF35F8F2000FFF7E9FF094B5C
:100CB000984201D0A84205D1320029002000FFF758
:100CC0004BFF70BD044B054A0548862101F0ECFA44
:100CD000240100D0CD010010285700103C5800100E
:100CE000A0560010F0B5CE46474680B583B006004A
:100CF0000D00EFF3108872B64F4B1B68002BFBD032
:100D0000BFF35F8F4D4B9A6834001034A300D7585F
:100D10004B4B9F4207D0AF4200D18BE00197494B2C
:100D2000FB1A2F2B09D9424639003000FFF714FF78
:100D300003B0C0BCB946B046F0BD3000FFF77CFF41
:100D4000814600213000FFF793FFBFF35F8FEFF381
:100D50000581002901D08C4211D10123019C9C43C3
:100D60000020A368AB4212D00622A256002A0DDB57
:100D700053009B189B00334A2000D418F1E7324BF4
:100D8000324A36213248FF3101F08EFA2000AB4260
:100D900049D106256557002D2BDB2A4B6A005219D5
:100DA00092009B189A68A260DA79E2719B795BB233
:100DB000A371002B0FDA2748A080224B6A0052193A
:100DC00092009B18244A1178997115704946300099
:100DD000FFF74EFFA7E7680040198000194BC018C5
:100DE0000430FFF7CDFE0100231D1800FFF7E0FEE1
:100DF000E2E7002912D100280ED0FF238371174BA0
:100E0000838015490B78A3710E4A154BA41A6441CF
:100E100063431B0D0B70D9E7094FF2E71149201D01
:100E2000FFF7EAFED2E7104B084A6A210848FF3173
:100E300001F03AFA024F76E7240100D000ED00E01D
:100E4000CD0100103C020020605700100C5800102B
:100E5000A056001001BD0000870D002001BDFFFF5E
:100E6000AAAA0000760200209457001070B5012253
:100E700002432E4BD31A2F2B28D8EFF30583002BD8
:100E80002BD0EFF3108C72B6294909680029FBD0EA
:100E9000BFF35F8F254C274905002D1B6D4169432A
:100EA000090D4CB2244989689B00C95891421BD056
:100EB0000021032932D81D4B4A00521892009B187A
:100EC0009B795BB2A3421FD00131F2E71B4B1C4A56
:100ED000C7211C48490001F0E7F91B4B184A922131
:100EE0001848FF3101F0E0F9134A92681749D150D0
:100EF000174B1A7882711C70BFF35F8F0C4B002266
:100F00001A608CF3108870BD084B4A005518AD006C
:100F10005D19FF26AE710F4AAA80E9E70E4B084A19
:100F2000D1210848490001F0BFF9C0463C02002029
:100F3000240100D0AAAA000000ED00E09C57001098
:100F4000D8570010A0560010C4570010CD01001053
:100F5000870D002001BDFFFFD05700100022044B79
:100F600002E0044902C30132072AFAD97047C04699
:100F700000E400E080808080024B9C466144890050
:100F8000016070474000003410B50400FFF7D6FD43
:100F900001002000FFF7F0FFFF232371BFF35F8FF5
:100FA00010BD10B50400FFF7C9FD01002000FFF7D8
:100FB000E3FFFF23237100236371BFF35F8F10BD35
:100FC000084B5B6A994209D8064A926A824207D264
:100FD000994201D0012002E0002000E0002070478B
:100FE0000120FCE70040054010B500290AD0036845
:100FF0001B7B8B4206D38068054B9C4661440901EC
:10100000401810BD034B044A04483C2101F04CF940
:10101000FFFFFF0F145900104C5C001038590010EE
:10102000F8B504001700FFF7DFFF066845683900D0
:101030002000FFF7D9FF026843680120AB4201D8C6
:1010400002D00020C0B2F8BDB242FBD8F9E70000E0
:1010500010B5002B02DB0260436010BD024B034A57
:1010600003483F2101F020F994550010185C00104E
:10107000B055001010B582B00400049805991218FC
:101080004B41002B09DB6846FFF7E2FF009A019B0A
:1010900022606360200002B010BD01225242014B69
:1010A000F1E7C046FFFFFF7F10B5002908D0037BA2
:1010B0008B4205D300684B005B18033BC01810BD82
:1010C000024B034A0348682101F0EEF87C590010F6
:1010D000F45B00109859001010B5437B8B4201D18E
:1010E000012010BDFFF7E0FF8378002B01D1002025
:1010F000F7E70120F5E770B50400857B002D01D1ED
:10110000280070BD2900FFF7CFFF4378A373002BA1
:1011100000D1E3730023837043700370F0E7000095
:10112000F8B506000C001500FFF7BEFF0700002C05
:101130000DD0002D11D0AC4215D029003000FFF7A2
:10114000B3FF84703B78002B13D13D70F8BD0A4B80
:101150000A4A0B486F2101F0A7F80A4B074A0848D2
:10116000702101F0A1F8084B044A0548712101F0F3
:101170009BF843703D70E9E7EC590010D05B00101C
:1011800098590010F8590010045A001070B5060064
:101190000D001400002914D0002A14D04368806880
:1011A0009847002806D0220029003000FFF7B8FF3A
:1011B000280007E02A0021003000FFF7B1FF2000DF
:1011C00000E0100070BD0800FCE7000070B50400EE
:1011D0000D1E0CD0FFF768FF00238370437003706F
:1011E000617B2A002000FFF7D1FF607370BD034BC5
:1011F000034A0448A52101F057F8C0461C5A0010C4
:10120000E45B00109859001070B504000D1E0FD05B
:10121000FFF762FF00280BD1E17B00290ED1A37BF1
:10122000002B03D1E37B002B0DD1A573E57370BDBB
:10123000084B094A0948F62101F036F82000FFF76B
:1012400033FF4570EBE7064B034A0448FB2101F0EE
:101250002BF8C046205A0010C05B001098590010AF
:10126000445A001010B5002907D003681B7B8B423D
:1012700003D3C0680139401810BD034B034A04482A
:10128000412101F011F8C04614590010AC5B001068
:101290003859001070B505000C00080000F092FCF1
:1012A0000949200000F0D2FBFFF748FC074B9C46A1
:1012B0006044800068602C75D0231B061B786B751A
:1012C000034BA400E55070BDE11300104000003452
:1012D000380B00200A4B1A68EFF3108172B61368BE
:1012E000002BFCD0BFF35F8F054B1B68BFF35F8FF4
:1012F00000221A6081F3108840BF0020002170474F
:101300004C0D002010B582B0040000F07FFB0200FD
:101310000B006846FFF79CFE009A019B2260636009
:10132000200002B010BD70B584B0040016001D008E
:1013300002A8FFF7E7FF029A039B009601952000A1
:10134000FFF798FE200004B070BD0000F0B583B038
:10135000070001921D000AAB1C780BAB1E78002C15
:101360000BD000682100FFF7B7FE002809D0194B09
:10137000194A1A48672100F097FF0068FFF7BBFE83
:101380000400002C02D1200003B0F0BD2100380081
:10139000FFF72AFE019B03604560089B8360099B61
:1013A000C36038682100FFF711FFA042EBD1387D00
:1013B000019A2B0000F092FB051E01D0002E04D0F4
:1013C0000C9B002BDFD01D70DDE73868210000F09A
:1013D0003FFDF5E7585A0010005C00103859001026
:1013E000F0B5DE4657464E464546E0B58FB00B9009
:1013F0000021784B8200D458894682E029002000E1
:10140000FFF7F2FD804602684368921BBB41002B48
:1014100009DD43461A685B680B9800F05FFB002308
:101420009846002689E0002B01D1002AF1D1002145
:10143000584600F003FD0700A84215D143461A683C
:101440005B680892099343469E68DB689846002EC5
:1014500010D029002000FFF705FF037899461B02F2
:101460001F432761002068E05B4B5C4A5C488E218B
:1014700000F01AFF5B4B594A5948922100F014FFC3
:101480002369002B77D0BB4219D106980799002316
:1014900042428B4100920193089A099B0CA8FFF7E6
:1014A000E9FD0C9A0D9B00210491013103910295F5
:1014B0004146019100962000FFF748FF16E04A4B95
:1014C000464A4748A12100F0EFFE069A079B002BF1
:1014D00001D1002A52D120682900FFF795FE29008A
:1014E0002000FFF7BFFE0378013303700023236160
:1014F0006268BFF35F8F13608AF3108801200028B1
:1015000061D00CA8FFF7FEFE0C9E0D9F0022002369
:10151000089209936268EFF3108A72B61368002B81
:10152000FCD0BFF35F8F23689B465D7B002D00D00E
:1015300064E700239846002600206368BFF35F8FAE
:1015400000221A608AF31088002ED8D04B461F0262
:101550002F4341463800B047069007916268EFF389
:10156000108A72B61368002BFCD0BFF35F8F079B05
:10157000002B00DA84E7079B002BA6DD2369002BF4
:10158000A9D0BB4219D10CA8FFF7BCFE0C9A0D9B49
:1015900006980799009001910CA8FFF76BFD0C9A33
:1015A0000D9B002104910131039102954146019167
:1015B00000962000FFF7CAFE98E70B4B074A084841
:1015C000A42100F071FE0FB0F0BCBB46B246A946A4
:1015D000A046F0BD380B0020805A0010305C00108F
:1015E00038590010985A0010A45A001010B50C4B2E
:1015F0005B68002B04D00B480A21FFF7BDFC10BD2F
:10160000074C094A20682300102100F082FB0320C8
:1016100000F0F0F903212000FFF73CFEEBE7C046A5
:10162000840200204C0D00202110001010B5064B44
:101630005B68002B01D0044810BD044B044A0548E8
:101640005E2100F031FEC04684020020E05A001006
:10165000945B001038590010F0B5DE4657464E46F0
:101660004546E0B58DB0060090461F00169B9A4691
:10167000179B994618AB1B780793272302AA944619
:10168000634400221A7021E001003000FFF7EAFDF8
:1016900000783CE00698002B5CD0079B002B59D0CB
:1016A0004946D04704000D0003000B4359D00029E0
:1016B00040DB08A8FFF726FE089A099B00940195D5
:1016C00008A8FFF7D7FC089B9846099F7268EFF3BC
:1016D000108B72B6136859424B41D9B20691002B58
:1016E000F8D1BFF35F8F273302AA94466344049373
:1016F0000023039302934B460193534600934246C3
:101700003B003000FFF722FE0400051EBCD17368C9
:10171000BFF35F8F002119608BF31088002D17D065
:10172000272302AA944663441B78002BB2D10002FF
:101730002043B0E700236242AB410092019342464E
:101740003B0008A8FFF796FC089B9846099FBDE759
:10175000012040420DB0F0BCBB46B246A946A046AF
:10176000F0BD0698F6E7F0B5C64600B584B00500B2
:10177000884616001F000AAB1C78FFF757FF02943B
:10178000019700962A004346FFF766FF04B080BC2D
:10179000B846F0BDF0B5C64600B504000D0042687D
:1017A000EFF3108772B61368002BFCD0BFF35F8F86
:1017B000EEB22368984631001800FFF78DFC002830
:1017C0002AD02369AB4213D02D0AEDB2310020009C
:1017D000FFF748FD0378AB4211D000206368BFF3E8
:1017E0005F8F00221A6087F3108880BCB846F0BD76
:1017F0000C4B0D4A95210D48490000F055FD310074
:10180000404600F025FB0028E8D1094B064A32216A
:101810000648FF3100F048FD2369AB42DED10023CA
:101820002361DBE7045B00107C5B0010385900107B
:10183000285B001010B50400FFF7F8FE2100FFF749
:10184000A9FF10BD30B587B004000D00EFF305838C
:10185000002B20D106225242D31712196B418B4222
:1018600002D803D1824201D90022002304A8FFF745
:10187000EFFB02A8FFF746FD02980399049A059B27
:10188000121A8B41002B0BDC08D02000290000F03D
:10189000C9F807B030BD144800F09EFD002AF4D00E
:1018A000124A0498059900230093FFF75CFF002873
:1018B00013DAEAE70E4B1A68EFF3108172B6136879
:1018C000002BFCD0BFF35F8F094B1B68BFF35F8F0A
:1018D00000221A6081F3108820BF04980599FFF751
:1018E0006FFB0028E6D0D0E72C5B0010D51200106B
:1018F0004C0D002000B583B002000B006846FFF7D6
:1019000012FD00980199FFF79DFF03B000BD10B5CF
:10191000FA2292000023002102F0ECFCFFF7EAFF1C
:1019200010BD000030B583B005000C00EFF3058357
:10193000002B0FD10B4A00230093FFF714FF002860
:101940000BDD20BFFFF776FF28002100FFF738FBF3
:1019500003B030BDFFF734FBFAE728002100FFF7A2
:101960002FFBF5E7D512001070B5EFF305801038A6
:10197000EFF3108C72B6194B1B68002BFBD0BFF332
:101980005F8F01221300834015494B6315490B609B
:10199000154909780C00C440224213D0104A546AF9
:1019A000124A8500AA58944205D3114AAA580E4CEF
:1019B0009943217007E00A4A031D9B0099589950EA
:1019C000002200E00022BFF35F8F044B002119606A
:1019D0008CF31088002A00D0904770BD280100D0F9
:1019E000004005403C700540880D0020500D00204F
:1019F000AC0A002010B50100024A034B1800FFF7A3
:101A00004BF810BD585C0010860D0020044B5B6A3B
:101A1000034A906A1900536A9942F9D17047C04647
:101A200000400540084B5B6A01E0074B5B6A8B4254
:101A3000FBD301E0044B5B6A8B4203D1024B9B6AF0
:101A40008342F7D37047C0460040054070B504009C
:101A50000E00EFF3108572B61B4B1B68002BFBD0FA
:101A6000BFF35F8F002E1CD02000FFF709F9174B42
:101A700083420BD019002000FFF70AF90121200052
:101A8000FFF7F6F80123A340114A1360114BA4009D
:101A9000E650BFF35F8F0C4B00221A6085F310886D
:101AA00070BD0C4BA2000021D1500122A2400A4976
:101AB0000B7893430B7005492000FFF713F90021C1
:101AC0002000FFF7D5F8E4E7280100D069190010DD
:101AD00038600540AC0A0020880D0020F0B5DE46D5
:101AE00000B584B00400150001921E000293FFF7B8
:101AF0008DFF03958E4202D84ED185424CD9EFF32B
:101B0000108B72B6274B1B68002BFBD0BFF35F8F87
:101B1000254A17780125A540EBB23B431370234BB0
:101B20005D63221D92000199D150214AA1000298C3
:101B300088501B6A2B4212D11C4B1B6C2B4208D0C5
:101B40000020BFF35F8F174B00221A608BF31088C1
:101B500023E0184B184A1948C52100F0A5FBFFF7F0
:101B600055FF8E4214D802D1039B834210D80E4BEE
:101B70001B78BB420ED00D4B1D625D631F222240BD
:101B8000012393400E4A1360074B1F700120D8E7D2
:101B90000020D6E70120D4E7012004B080BCBB467A
:101BA000F0BDC046280100D0880D0020004005404F
:101BB000500D00207C5C0010EC5C0010A05C00105C
:101BC00080E200E0EFF3108C72B60B4B1B68002B29
:101BD000FBD0BFF35F8F01238340084A136208499B
:101BE0000A789A430A70BFF35F8F034B00221A6092
:101BF0008CF310887047C046280100D00040054093
:101C0000880D002010B5002908D0037B8B4205D336
:101C100000684B005B18033BC01810BD024B034A21
:101C20000348682100F040FB7C590010005E001062
:101C300098590010F8B506000C001500FFF7E2FFF8
:101C40000700002C0DD0002D11D0AC4215D029007A
:101C50003000FFF7D7FF84703B78002B13D13D7025
:101C6000F8BD0A4B0A4A0B486F2100F01DFB0A4BD6
:101C7000074A0848702100F017FB084B044A054842
:101C8000712100F011FB43703D70E9E7EC59001041
:101C9000EC5D001098590010F8590010045A00101B
:101CA00070B506000D001400002914D0002A14D0CD
:101CB000436880689847002806D022002900300039
:101CC000FFF7B8FF280007E02A0021003000FFF7E7
:101CD000B1FF200000E0100070BD0800FCE770B507
:101CE00005000023437301338373037BC373012413
:101CF00006E021002800FFF785FF0134E4B24470BC
:101D0000297BA142F5D82800FFF77CFF0023437010
:101D100070BD10B5017342608360FFF7E0FF10BD36
:101D2000F0B5C64600B505000C1E03D1200080BCEE
:101D3000B846F0BDFFF766FF4678002EF6D03100BA
:101D40002800FFF75FFF4778002398464370210083
:101D50002800FFF757FF4346437032002100280058
:101D6000FFF79EFF040039002800FFF7D9FF0200AB
:101D700021002800FFF794FF0400D7E7F0B5C6461E
:101D800000B504000D001700002927D0FFF73AFF27
:101D90004378002B28D18378002B2BD101782000A9
:101DA000FFF7BEFF06008046002F0AD0E17B002926
:101DB00026D1A37B002B03D1E37B002B25D1A57378
:101DC000E5734346002B26D129002000FFF71AFFB8
:101DD00000234370300080BCB846F0BD114B124A5E
:101DE0001248382100F060FA114B0F4A0F483A218F
:101DF00000F05AFA0F4B0C4A0C483B2100F054FA01
:101E00002000FFF7FFFE4570D3E70B4B064A07485B
:101E1000422100F049FA31002000FFF7F3FE0023D1
:101E20008370D1E7085D0010D85D0010105D0010D0
:101E3000545D00107C5D0010445A001070B5040021
:101E40000A00457B2900FFF799FF6073280070BDE9
:101E500070B506000C1E40D0437B8B4207D0FFF7C5
:101E6000D1FE05008178002906D1002036E001214D
:101E7000FFF7E4FF012031E03000FFF7C3FE0178F7
:101E8000A1420DD03000FFF7BDFE4178A1420AD03B
:101E90000029F7D1124B134A13486B3100F004FAB2
:101EA0006B78037001E06B7843700023AB706B704C
:101EB000012221003000FFF761FF0200717B8142A7
:101EC00005D03000FFF7ECFE7073012006E0074BF1
:101ED000044A0548712100F0E7F9002070BDC046B2
:101EE000D0570010C05D0010105D0010A05D001004
:101EF000F8B5DE4657464E464546E0B506000F00AB
:101F000015000A9A93424ED31A0E92461B02984627
:101F10000A9A00234046514601F0ECFB81467400CA
:101F2000A419A4002E4B9C4664446368834200D2EB
:101F30006060331FDBB29B46012B3AD9C0239B0163
:101F40002343802212011A60264BB200D158002987
:101F500005D0586901F090FB01300138FDD16D01C9
:101F600023685D40E0222A4080235B0123431A60FE
:101F70005A46012A28D980239B012343802212013B
:101F80001A604B4663604A4600234046514601F0C2
:101F9000B1FB144BB60098510120F0BCBB46B246D1
:101FA000A946A046F8BD104B104A11482D2100F05B
:101FB0007BF9012FC2D1C0239B01234303221A6066
:101FC000A368DB07FCD5CAE72168794003220A40F1
:101FD0001A60A3680125BD401D42FAD0CBE7C04678
:101FE00000800040BC0A00200C5E0010705E0010F3
:101FF000205E001030B583B00C2000F017F9FEF71A
:102000002BFD00280DD0002304E02E4A99002E4815
:1020100088500133092BF8D92A4B2C4A5A6203B055
:1020200030BD2B4B00229A6700F008F9294B0122A2
:102030001A60274B5B6C012BFBD1274B03221A60E4
:10204000234B9B6B012BFBD1013300930433234AB9
:102050000121234800F054F805230093214A01216F
:10206000214800F04DF8214B00930022022104206A
:10207000FFF73EFF1E4D00952B0000220121052099
:10208000FFF736FF104C00942300002200210720A8
:10209000FFF72EFF00942300002200210820FFF705
:1020A00027FF0A4B00932300002200210920FFF79D
:1020B0001FFF00952B00002200210620FFF718FFCC
:1020C000ADE7C046BC0A0020006CDC021BB7000074
:1020D000008000403CB0004030B00040002F685904
:1020E00000800240008C864700C00240001BB70001
:1020F00040597307014B8000C0587047BC0A00204C
:10210000F0B5C64600B504000D00170098460C2037
:1021100001F0B2FA0600394BFA18394B9A4241D80D
:1021200043011B1A9901C91AC9000918890138000D
:1021300001F0A2FA0200103A98235B009A4237D8C5
:102140004346013B062B39D8069B013B062B35D86D
:102150003F09B74238D343461E04069B1B031E4368
:102160002368002B36DB274B9C4244D080235B0145
:10217000254A1360254A1360254A92681900914345
:10218000FAD12560A060221DC0239B0113432122A8
:102190001A602268002AFCDAE66008221A6080BC15
:1021A000B846F0BD1B4B1C4A1C48112100F07CF8BE
:1021B0001B4B194A1948192100F076F8194B164A99
:1021C00016481C2100F070F8174B134A13482321BE
:1021D00000F06AF822683F231340AB42C3D1A368E2
:1021E0001B051B0D8342BED1E368EE22D2021340D1
:1021F000B342B8D1D3E780239B01B9E780E84BD342
:1022000080F8A93200C0024000E0004000F0004029
:1022100000C00040805E0010AC5F0010E05E001067
:10222000285F0010445F0010905F001080239B0027
:102230000343014AD362704700800540064BAA223F
:1022400012011A602F22DA60044B054A1A60024B11
:102250005B68002BFBDA70470040024000600240E0
:1022600000B0FA0000BEFDE703000A4A1268002A27
:1022700008D0084A1068C318074A9A4206D3054A8C
:1022800013607047034A05491160F2E7012040429C
:10229000F7E7C046340B0020000004208C0D00201E
:1022A00010B5FFF7DFFF000030B583B00D00190057
:1022B000002A0BD0074B084C019200932B00020020
:1022C000200002F0CBFA0120FFF7CCFF034B1A00ED
:1022D000F1E7C046B85F0010C85F0010C45F00108F
:1022E00070B52B4B2B4A1A602B4B2C4A1A602C4B87
:1022F0009A682A4B9343FAD12A4C01E008CC9847BC
:10230000294B9C42FAD3FFF775FE234B274A1A60EC
:10231000234B9B68DB43DB01FAD1254B40229A67B4
:102320005A671A67DA66234C09E0234B234A24488C
:102330008621FFF7B9FF2000FEF726FE0834214B67
:102340009C4209D22368002BF5D0012BEDD120004F
:10235000FEF727FE0834F2E71B4DA9681B4CC0228C
:10236000200002F001F9AC60EFF30583002B00D0F0
:1023700000BEFEF7D3FBFEF7F1FDFFF737F9144C73
:1023800001E008CC9847134B9C42FAD370BDC0467D
:1023900000E00040BFCDFBFE00F00040FE7F3C00AF
:1023A00000C000401008002020080020FFFFFF01AF
:1023B00000F0014008080020F85F0010786000106D
:1023C000186000101008002000ED00E00000002060
:1023D00020080020240800200FB400B583B008486E
:1023E00002F00CFA049B002B07D005A901911800FC
:1023F00002F014FA034802F001FA0120FFF732FF5D
:102400006460001074600010704710B5002802D09E
:102410000B684968984710BD0100002007E0830061
:102420001B185B00501C08601078C01830380A6810
:102430001378303BDBB2092BF1D97047F0B5DE469B
:1024400057464E464546E0B583B093461F000C9B69
:102450009A460D9C0E9B99460F9B9B0703D0B8464E
:102460000F00060022E00192A34688464E46B94678
:102470000700B44207D2551C4B4641462020B847BE
:1024800001342A00F5E73D004F465C46019B9B4620
:10249000B1464646B84637002E0007E0013C551CC1
:1024A0005346185D43463900B0472A00002CF5D149
:1024B00035003E0047460F9B9B0707D4100003B032
:1024C000F0BCBB46B246A946A046F0BDB0464E465B
:1024D000B9462F005D46531BB342EFD2541C4B4606
:1024E00041462020B8472200F5E7F0B5CE464746E2
:1024F00080B585B0944698460C9D0D9C0EAB1B781C
:102500009946109A119B129EB7071CD4002B0CD031
:10251000F7070AD54F46002F02D10C37374204D0B7
:10252000013B02E030272F550134944201D21F2C89
:10253000F8D9F70707D59C4205D21F2C03D83027BE
:102540002F550134F5E7F70612D5770505D4002C91
:1025500003D0944221D09C421FD00F9A102A32D02F
:102560000F9A022A37D01F2C0AD830222A5501345C
:102570001F2C05D84A46002A33D02D222A55013473
:10258000039602930194009543466246FFF756FF77
:1025900005B0C0BCB946B046F0BD621E012C10D0DB
:1025A0000F9F102F0BD014000F9A102AD8D1B2060B
:1025B000D6D51F2CD4D858222A550134D3E7023C53
:1025C000CBE71400C9E7B206EED41F2CECD8782272
:1025D0002A550134C7E71F2CD2D860322A5501345E
:1025E000C1E7720703D52B222A550134C8E7320709
:1025F000C6D520222A550134C2E7F0B5DE4657463B
:102600004E464546E0B593B081468A460892099306
:102610001CAB10CB1B789B461E9D219B9846002C23
:1026200003D1102342469A4390468023DB0046465E
:102630001E4042461A4212D0002C22D000260EE044
:102640003033D9B2771C0AAB99552900200001F02C
:1026500013F8AC4216D31F2F14D83E0004002900F3
:10266000200001F009F8CBB2092BE9D942469206C5
:1026700005D54121C918C9B20A39C9B2E2E76121B9
:10268000F8E7270043460693209B05931F9B04937E
:1026900003955B46029301970AAB0093099B089A46
:1026A00051464846FFF721FF13B0F0BCBB46B24687
:1026B000A946A046F0BDF0B5DE4657464E46454613
:1026C000E0B597B00A900B910C929A46209B9946E0
:1026D000219F22AA13789B46249B0993259C289B23
:1026E00098464A463A4302D1103293439846802294
:1026F000D20045461540434613420AD04A463A4363
:1027000041D000252E0053460D934D46099B9A4615
:102710001BE02E0053460D934D46099B9A4614E04C
:102720003033DAB2731C99460EAB9A5552462300E9
:102730002800390000F0DEFFBC4226D819D04B46F5
:102740001F2B1CD84E4605000F00524623002800C0
:10275000390000F0CFFFD3B2092BE1D942469206EF
:1027600005D54122D218D2B20A3AD2B2DAE76122B2
:10277000F8E7AA45E3D94E460D9B9A4608E04E4637
:102780000D9B9A4604E0002602E04E460D9B9A46B9
:1027900043460693279B0593269B0493099B03932B
:1027A0005B46029301960EAB009353460C9A0B992D
:1027B0000A98FFF79AFE17B0F0BCBB46B246A9468E
:1027C000A046F0BDF0B5DE4657464E464546E0B55C
:1027D00091B0804689460C929A461A9C1B9D220015
:1027E0002B002000290001F010FA002800D0ECE0B6
:1027F00001225242D44B2000290001F001FA0028A6
:1028000000D0E2E001225242D04B2000290001F02A
:10281000E1F9002800D0D8E00022002320002900A0
:1028200001F0D8F9002800D0E4E006940795802351
:10283000DB001E9A1A400D921E9A1A4201D10623FD
:102840001C930698079902000B0008920993030055
:102850000A00024300D1D9E0080D4005400DBC4EEE
:10286000B44660440A03120B1E00BA4B13431F0008
:1028700001F0DEF9B84AB94B01F069F9B84AB94B31
:1028800001F03EF9089009910022B74B3000390061
:1028900001F02DF9B54AB64B01F059F902000B00D1
:1028A0000898099901F02CF901F0DAF9834601F052
:1028B000BFF906000F00AF4AAF4B01F048F9002204
:1028C000AE4B01F01DF901F0CBF90890AC4AAD4BCD
:1028D0003000390001F03BF906000F00089801F0C4
:1028E000A7F9A94AA94B01F032F902000B00300008
:1028F000390001F0FCF806000F0002000B0001F0A7
:1029000026F90A900B91089BA14A94466344002142
:102910000022089109921B050993002308933200B5
:102920003B003000390001F0EBF80E900F913200BF
:102930003B0000208021C90501F0D9F806000F00F6
:102940000022944B0A980B9901F0E3F80022924B75
:1029500001F0D6F802000B000A980B9901F0D9F8A3
:1029600000228E4B01F0CCF802000B000A980B9964
:1029700001F0CFF802000B003000390001F0C0F880
:1029800002000B000E980F9901F0C3F80022714B62
:1029900001F0B6F8089A099B01F0D9F806000F007B
:1029A00008960997069A079B01F02AF900282FD06C
:1029B00001235B429C46E3440022774B3000390000
:1029C00001F0A7F80890099122E01E9B04931D9B3B
:1029D00003931C9B02930094019553460C9A49461D
:1029E000404600F0FFF811B0F0BCBB46B246A94625
:1029F000A046F0BD00210022069107920694802394
:102A00001B069C46AC446346079310E700239B4695
:102A10005B466333C62B20D804261E9B1B0528D596
:102A2000089A099B190011430FD05D4A5D4B069827
:102A3000079901F0DDF800287AD000225A4B069859
:102A4000079901F0C7F8002872D01C9B5B4506DD92
:102A50005A469B1A013B1C9303E00526DDE7002341
:102A60001C938023DB001E9A1A431E92002600232B
:102A70009B461D9B9E4265D29F1B02231E9A1A40B5
:102A80000A921E9A134202D0002E00D000275B4605
:102A9000002B07D0089A099B0698079901F039F88E
:102AA00006900791002200232000290001F092F8EF
:102AB000002800D07CE03D4B1E9A134004930397FE
:102AC0001C9B0293069B079C0093019453460C9A0F
:102AD0004946404600F086F8002E00D183E71E9B51
:102AE0009B0671D54525441C5346020049462800E3
:102AF000C0475A46D317D2185A4005230593013EC2
:102B00000496002303930A3302935B46DB0F019381
:102B100000925346220049464046FFF76EFD0A9B4D
:102B2000002B00D15FE7020047460C9E1D9D53E03D
:102B30001C9B002B9DD00D9B002B9AD01C9B013B16
:102B40001C9396E7002798E7FFFFEF7FFFFFEFFF5B
:102B500001FCFFFF0000F03FFB799F501344D33F7F
:102B6000B3C8608B288AC63F0000F83F61436F639B
:102B7000A787D23F71A379094F930A400000E03F35
:102B80001655B5BBB16B0240EF39FAFE422EE63F57
:102B9000FF03000000002C4000002440000018400B
:102BA0002D431CEBE2361A3F80842E41FFF7FFFFD6
:102BB000069C079D2200290080200006844661446F
:102BC0000B000692079376E765258CE7541C534665
:102BD00049462020B8472200931BAB42F6D3100091
:102BE00001E7C046F0B5DE4657464E464546E0B5DD
:102BF00095B00690079193469946209F1E9A1F9B79
:102C00001000190001F001F8002831D101225242D0
:102C1000BF4B1E981F9900F0DDFF002837D101221D
:102C20005242BC4B1E981F9900F0EAFF00283DD18C
:102C30000022B94B1E981F9900F0E2FF002850D1E6
:102C40000022B64B1E981F9900F0C4FF002848D1FF
:102C5000002200231E981F9900F0BCFF002850D1CD
:102C600000239846229B5B0500D4B6E0002458E080
:102C7000229B0393219B029303230193A84B009370
:102C80004B465A4607990698FFF7D8FB0EE1229B60
:102C90000393219B029304230193A24B00934B4681
:102CA0005A4607990698FFF7C9FBFFE00423229ACA
:102CB0001A4022990B4210D09B4B002A0FD00422BD
:102CC0002299039121990291019200934B465A4611
:102CD00007990698FFF7B2FBE8E0944BEDE7032273
:102CE000EEE7229B0493219B039302971E9B1F9C5C
:102CF000009301944B465A4607990698FFF762FDE8
:102D0000D4E01E9A1F9B0020002100F0F0FE1E90D0
:102D10001F9101239846A5E70CAB30221A55013FBD
:102D200001341F2C01D8092FF6D81E981F9900F0E6
:102D300097FF050000F07CFF02000B001E981F9912
:102D400000F0D5FE7A4BFA009B181A685B680A926D
:102D50000B9300F0FCFE0890099100F0A5FF06001F
:102D600000F062FF02000B000898099900F0BFFE16
:102D70000890099100226F4B00F042FF00282ED0EE
:102D80000136300000F050FF02000B000A980B994A
:102D900000F026FF002801D001350026002F2CD19D
:102DA000280000F045FF02000B001E981F9900F05C
:102DB0009EFE06000F0000225E4B00F00BFF002875
:102DC00046D100225B4B3000390000F019FF00288B
:102DD0003ED1EB073CD501353AE0062746E7002215
:102DE000544B0898099900F0F5FE0028D6D1002E22
:102DF00001D0F307D2D50136D0E7AA461F2C11D84F
:102E0000013F0A21300000F037FC651C30310CAB6B
:102E100019550A21300000F02FFC092E0ED90600AA
:102E20002C00EBE755461F2C0CD87B1E002F09D039
:102E30000CAA302111551F000134F4E72B00554630
:102E40001C00F0E71F2C03D80CAB2E221A550134BE
:102E50001F2C10D80A21280000F0E6FB661C303138
:102E60000CAB19550A21280000F0DEFB051E01D02D
:102E70003400EDE734000323229A1340012B1CD0C9
:102E80001F2C06D84346002B32D00CAB2D221A55EE
:102E90000134229B0393219B029301940CAB00937A
:102EA0004B465A4607990698FFF7C8FA15B0F0BC8A
:102EB000BB46B246A946A046F0BD219B002B13D0CD
:102EC0004346002B02D10C3313420FD0219B013B10
:102ED0002193190003E00CAB30221A5501348C42C7
:102EE000CED21F2CF7D9CBE72199F8E72199F6E745
:102EF000229B5B0704D50CAB2B221A550134C8E783
:102F0000229B1B07C5D50CAB20221A550134C0E704
:102F1000FFFFEFFFFFFFEF7F65CDCD4165CDCDC159
:102F2000946000109860001088600010906000109D
:102F3000406200100000E03FF0B5DE4657464E46C6
:102F40004546E0B593B082468846934611930029E2
:102F500000D10DE300255646119B1878002800D1BA
:102F600009E3252809D06C1C5B462A004146B0477E
:102F7000119B013311932500EEE7013311930027D4
:102F800020E001231F4301321192012418E00223A3
:102F90001F4301321192012412E004231F43013226
:102FA000119201240CE008231F43013211920124E5
:102FB00006E010231F4301321192012400E0002497
:102FC000002C09D0119A1378203BD9B21029F6D8D9
:102FD0008B00C849CB589F46119B1A781300303B91
:102FE000DBB2092B10D92A2A13D00B94119B1A7823
:102FF0002E2A1ED0119A1378683BD9B2122959D8BB
:103000008B00BD49CB589F4611A8FFF705FA0B90DE
:10301000ECE71C9B1A1D1C921B68002B04DB0B9316
:10302000119B01331193E1E7022217435B420B939B
:10303000F6E78022D20017435A1C11925A781300E7
:10304000303BDBB2092B0BD92A2AD3D11C9B1A1D8A
:103050001C921C68002C08DB119B01331193C9E7FB
:1030600011A8FFF7D9F90400C4E70024F4E780238E
:103070005B003B43511C119151786C2901D01F001A
:1030800018E0C0239B001F430232119212E08023FC
:103090003B43511C11915178682901D01F0009E070
:1030A000C0231F430232119204E080235B001F43C0
:1030B00001321192119B1878672818D8252800D260
:1030C0004CE20300253BDAB2422A00D946E29300E3
:1030D0008A4AD3589F4680239B001F430132119296
:1030E000E8E780235B001F4301321192E2E7782872
:1030F00000D933E2692800D230E20200693AD2B244
:10310000012393407E4A134211D11A0600D500E2F2
:103110005B0500D422E21C9B1A1D1C921B689A4678
:10312000002C00D0B2E10122524253468EE16F28BA
:103130000ED006D858283DD0622804D102239C46E0
:1031400008E0782839D010239F43063B9C4601E0D5
:1031500008239C46582833D0692803D0642801D01E
:103160000C2297437A0501D50122974369282AD07A
:10317000642828D0BA0500D59FE0FA0500D5C1E043
:103180007A0600D4D3E01C9A111D1C911168FF220D
:103190000A4005970B9B0493039463460293002314
:1031A000019300925B462A0041463000FFF725FA62
:1031B000050027E010239C46CCE710239C46C9E776
:1031C00020221743C8E7BA0520D4FA0550D47A065E
:1031D00066D51C9A111D1C911168FF220A40D01758
:1031E0001118414005970B9B049303946346029387
:1031F000D20F019200915B462A0041463000FFF752
:10320000FCF90500119B01331193A5E61C9A0732C6
:1032100007218A43110008311C91116853689946AF
:10322000DB170C930D930C9A0D9B100048400E90E9
:103230004A4653400F930E980F990C9A0D9B801A93
:1032400099410E900F9108970B9B07930694634644
:103250000493002305934B46DA0F029200900191EC
:103260005B462A0041463000FFF725FA0500C9E712
:103270001C9A111D1C911268D01711184140059716
:103280000B9B0493039463460293D20F0192009127
:103290005B462A0041463000FFF7AFF90500B1E771
:1032A0003A0605D51C9A111D1C910023D25E96E7A3
:1032B0001C9A111D1C91126891E71C9A0732072174
:1032C0008A43110008311C9108970B9B07930694C1
:1032D0006346049300230593029353681268009297
:1032E00001935B462A0041463000FFF7E4F90500F0
:1032F00088E7C046A0600010E46000103061001054
:10330000419000001C9A111D1C9105970B9B049382
:1033100003946346029300230193136800935B4672
:103320002A0041463000FFF768F905006AE73A06CF
:1033300006D51C9A111D1C9112681204120C28E764
:103340001C9A111D1C91126823E7462819D01C9B5A
:103350000733072293431A0008321C9204970B9AF2
:10336000039202941A685B68009201935B462A00FC
:1033700041463000FFF736FC0500119B01331193E5
:10338000EAE520231F43E2E7672801D0472802D15E
:1033900080231B011F43452801D0472801D120234A
:1033A0001F431C9B0733072293431A0008321C92C9
:1033B00004970B9A039202941A685B680092019337
:1033C0005B462A0041463000FFF7FCF90500119BDF
:1033D00001331193C0E502231A003A4091463B4263
:1033E0001DD001241C9B1A1D1C926F1C18785B4673
:1033F0002A004146B0474B46002B14D1119B0133A4
:1034000011933D00A8E5571C5B4641462020B0477C
:1034100023003A005C1C9D42F5D81500E2E7012329
:103420002A000B9DF6E73A00B1460B9E06E0571CBA
:103430005B4641462020C8472C003A00651CA64246
:10344000F5D817004E46D9E701330A00197800294C
:1034500002D0511E002AF7D152469B1A8022D20078
:10346000390011408946174202D0A34200D92300F7
:1034700002221100394010913A4209D02A00250059
:1034800057469A4633004E46994621E022004CE6C4
:103490002A004546A04606E0541C5B462900202031
:1034A000B0473B0022005F1C0B999942F4D8444678
:1034B000A8463B00250057469A4633004E4699469B
:1034C00006E01D000137541C5B464146C8472200F8
:1034D0003878002804D0002EF4D06B1E002DF0D1D7
:1034E000150053464E46109A002A03D1119B013312
:1034F000119331E50B9F2A0006E0551C5B464146BF
:103500002020B04723002A005C1C9F42F5D81500FC
:10351000ECE721233B431C9A111D1C911268059373
:103520000823049303940833029300230193009229
:103530005B462A0041463000FFF75FF80500119B0B
:103540000133119308E56C1C5B462A004146252097
:10355000B047119B013311932500FDE46C1C5B46C1
:103560002A004146B047119B013311932500F3E433
:103570000A4B9A46EEE4B2465D450DD35B465A1EB1
:103580005B4641460020D047280013B0F0BCBB4644
:10359000B246A946A046F0BD2A00F1E70924001072
:1035A00000B585B0029003910121044800931300F7
:1035B0004A4202A9FFF7C0FC05B000BD0B24001071
:1035C00001480421014B1847B0020020F1350010DA
:1035D00010B5010018231B8814221088984710BDCD
:1035E00010B5010018231B8816221088984710BDBB
:1035F000F0B5C64600B507000E0000250123984629
:1036000000E00135B5420AD2AC003C192068FFF752
:10361000DFFF20600028F4D100239846F1E7404600
:1036200080BCB846F0BD0000124A936F9B0815D2CB
:103630009066D166002905D0FFE7FFE7FFE7516FED
:10364000106F704704B580210906C2175140002849
:1036500000D0C84301F038FF002104BDF0B5146E5E
:10366000556E576F166FFFF7E3FF14665566576781
:103670001667F0BD000000D0114A936F9B0813D26B
:1036800010665166002905D0FFE7FFE7FFE7516F9D
:10369000106F704704B5002801D00020C04301F02E
:1036A00013FF002104BDC046F0B5146E556E576F70
:1036B000166FFFF7E5FF1466556657671667F0BD8E
:1036C000000000D094464A4A926F9208624601D2A6
:1036D00028E0C046F0B5464E346E756E776F366F93
:1036E00000F020F89446424A1466556657671667FC
:1036F0006246F0BD94463E4A926F9208624601D2FD
:1037000054E0C046F0B53A4E346E756E776F366F42
:1037100000F04CF89446364A1466556657671667AB
:103720006246F0BD002B24DB11D000293EDA00B543
:10373000C943404200D1013100F038F8C94340424A
:1037400000D10131DB43524200D1013300BD002AD8
:10375000EBD1002801D1002905D00020C90FC907ED
:1037600001D1C043410800B501F0A6FE00220023AC
:1037700000BD00B500290ADBDB43524200D1013312
:1037800000F014F8C943404200D1013100BDC943E3
:10379000404200D10131DB43524200D1013300F0FD
:1037A00005F8DB43524200D1013300BD002923D18B
:1037B000002B18D1002A0CD0BC460D4F38667A6613
:1037C00000210023FFE7FFE7FFE77A6F386F6746C6
:1037D0007047002801D00748010000B501F06CFED9
:1037E0000022002300BD02000B00002000217047D2
:1037F000000000D0FFFFFFFF002B00D0BFE0130C44
:1038000028D1002AE7D080B4114F39667A66FFE7E5
:10381000FFE730B4040C7B6F396F1B0423433B6616
:103820007A66FFE7FFE7FFE7C04684B27B6F3D6F34
:103830001B0423433B667A66FFE7FFE7C04600238D
:103840002C042D0C7A6F386F00196941B0BC704799
:10385000000000D0F0B594460025140E01D11202EC
:103860000835140F01D112010435940F01D19200D3
:103870000235D40F01D152000135D40B0134254F4C
:103880007C66254C3C660E0C93B2FFE7FFE7FFE732
:103890003C6F6643360C7703BE467343DF0B5B0415
:1038A000C01AB941130C7343DB18C91ACE0866431A
:1038B000360CB64493B273431F0F1B01C01AB941B3
:1038C000130C73431F0B1B05C01AB941860D8F02E1
:1038D0003E436643360C092D24DB520A7243801A9C
:1038E0007703460A6643360C16235B1BDE40DF4037
:1038F000BF1964466643821B7046043506330100D7
:10390000D940A840C01900D30131A24206D20023F9
:10391000F0BD0000000000D0FFFFFFFF121B0130D0
:10392000F3D3F1E709277F1BFE406446A2B272433E
:10393000801A00D20139220C7243130C1204821A2D
:1039400099410B007046043513370100F940A84037
:10395000801900D30131002B02D1A2420AD2F0BD5E
:10396000013000D30131121BFAD2013BF8D1A2423F
:1039700000D2F0BD013000D30131121BF7E7F0B5E2
:103980001C0C00D080E00CB400251C0A04D11B02E2
:10399000160E3343120208351C0B04D11B01160FFF
:1039A0003343120104359C0B04D19B00960F334323
:1039B00092000235DC0B02D192185B4101351C00EC
:1039C000971864410134464F7C66464C3C660E0CA9
:1039D000FFE7FFE7FFE7C0463C6F6643360C77031F
:1039E000BE4697B27743C01B00D20139C01B00D23C
:1039F00001399FB27743C91BC91B170C77437E045B
:103A0000FF0B801BB941CE086643360C0C2D33DB0F
:103A1000B644120B1F053A431B0B97B27743C01BEA
:103A200000D201399FB27743C91B170C77433E047C
:103A30003F0C801BB941860D8F023E436643292708
:103A40007F1BFE400C3D7746AF40BF1930BCA2B291
:103A5000ABB272437343801A9941220C7243130C28
:103A60001204801A994102000B000137001BA94182
:103A7000F9D2781E0021F0BD0C277F1BFE4077464F
:103A80007F0BAF40FF19E0E700245D1C07D0144F07
:103A90007D663966FFE7FFE7FFE7FFE73C6F95B21A
:103AA0009EB265436643401BB141150C1E0C654335
:103AB000664336042F0C3E432D04401BB14199420E
:103AC00004D202000B0020000021F0BD01D1904281
:103AD000F7D3801A994101349942F2D3F6E70000F6
:103AE000000000D0FFFFFFFF48404140484018B4AD
:103AF0001B4B5B68FC46019308BD04DFC73D00100B
:103B000018B4174B1B68FC46019308BD00DFD13D7C
:103B100000109446134A926F920809D2624618B474
:103B20000F4BDB68FC46019308BD0CDF8940001099
:103B30000C4AF0B5146E556E576F166F6246FFF75C
:103B4000EEFF084A1466556657671667F0BD18B44D
:103B5000034B9B68FC46019308BD08DF2D3F001016
:103B6000480B0020000000D0FFB5504042405040BC
:103B700059404B40594000E0FFB5154F4C00640DD3
:103B800003D0BC4204D10C0314D80020090D090550
:103B90005C00640D03D0BC4204D11C030AD800228F
:103BA0001B0D1B0501264B4009D44B4003D58B420E
:103BB00000D18242FFBD9942FCD19042FFBD0B4330
:103BC000DB1803431343F5D0C9434918FFBD000078
:103BD000FF07000000B5FFF7CFFF804100BDC046E2
:103BE00000B5FFF7C9FF01D9002000BD012000BDCD
:103BF00000B5FFF7B9FF01D9002000BD012000BDCD
:103C000000B5FFF7B1FF804100BD012040054A002B
:103C1000121804D85A00121801D800207047012049
:103C200070470020704700000021002805D1704730
:103C3000C1174840401AFAD0C90713B5064B1B6894
:103C400098470CBC441CA2401005120B0349091BE9
:103C500009051943114310BD480C00201F04000042
:103C600010B54C00620D8023D218DB00D21A5B0520
:103C70007E2A10DD9E3A13DACC170903490819434E
:103C80005242D140640001341532202A05DAD04076
:103C90000843604310BD002010BD0846604310BDBE
:103CA000C80FC018013810BD18B4044B5B6AFC463D
:103CB000019308BD24DF394200100000480B0020AA
:103CC00070B513231C78012C12D0012C12DC214B6F
:103CD000214A93642148FFF77BFC214B186070BD9B
:103CE0001C491D4A9800815001331F2BF8D9ECE77D
:103CF0000023FAE71B48FFF773FC05001A48FFF79B
:103D00006FFC023803789B007F2B09DD124880226C
:103D1000290000F029FC022C08D0022CDADCD6E7BE
:103D2000124B134A13483221FEF7BEFA124B1A887F
:103D3000B5231B029A4209D1104B1A88104B9A42A4
:103D400004D1104B1A88104B9A42E6D00020FEF79F
:103D500043FBC0468D3D0010480B00204C33000053
:103D6000480C0020534400005346000090620010AD
:103D700044630010F062001054380000D83800008E
:103D8000494600009C3800005946000007B56046CF
:103D9000002800D100BE01880A0A0230DF2AFAD1C9
:103DA000C9B2820804D3028840880004104300E0AE
:103DB0000068024A5050039007BD0000480B0020E5
:103DC0000FB403BC0CBCF0B50124E407634000E071
:103DD000F0B50C0DCF0F661E3605891B640503D3A5
:103DE000C943404200D30131640D03D0661CF60A7A
:103DF00007D0E41B00207F00791C89078912803CD2
:103E000024031D0DDF0F6E1E36059B1B6D0503D3AE
:103E1000DB43524200D301336D0D03D06E1CF60A12
:103E200007D0ED1B00227F007B1C9B079B12803D6F
:103E30002D032F1B661B58D4A446202E46DA2037AC
:103E40001400BC401D00BD40F24033412A4380189D
:103E50005941CB0F05D0C943C043002264425041B1
:103E6000514162464D0D28D10D0D07D100281FD0BC
:103E7000241940414941013A0D0DF9D0640006D39F
:103E8000013000D30131002C01D140084000013A3B
:103E90000BD4941CE40A04D112051144DB07194425
:103EA000F0BDD907204B194300E0D9070020F0BD31
:103EB0000029DDD1002CDBD1F0BD0132C60740085E
:103EC000CD0728434908002EE1D0D9E73C2E29DA56
:103ED000203E40371400BC4000D00124F24014437F
:103EE0001A00BB401C43D317ACE7AC46202F08DABE
:103EF00020360400B4400D00B540F8403941284355
:103F0000A5E73C2F0CDA203F40360400B44000D037
:103F10000124F84004430800B1400C43C117EAE70C
:103F200010001900002494E70000F07FF0B50C0D9C
:103F3000661E3605891BE60A6405640D02D0651C01
:103F4000ED0A04D0002001210905803C2403A44689
:103F50001C0D671E3F05DB1BE70A6405640D02D0DC
:103F6000651CED0A04D0002201231B05803C2403BC
:103F70007740644497B484B296B27443070C7E438E
:103F8000150C6F4380B26843361802D30120000439
:103F90003F183004350C00197D41844688B29AB22E
:103FA00050430C0C62431F0C7C438EB27E4392192B
:103FB00002D301263604A4191604170C36186741DB
:103FC00001BC81B29AB25143040C62431B0C5C43A6
:103FD00080B25843121802D30120000424181004A0
:103FE000130C401863412D185E410020474106BC68
:103FF00088B293B258430C0C6343120C544389B2F9
:1040000051435B1802D301210904641819041A0CE6
:10401000091862416D1856410020474118BCF90249
:10402000720D1143F0026A0D1043ED020A0D03D127
:104030006D1940414941013B124E9B1B7600B34232
:104040000ED26D0007D3013000267141664635431C
:1040500001D1400840001B05C918E4072144F0BD08
:104060000BDA013306D1013004D101314F0D01D0FB
:104070004908F2E7E1070020F0BD013631050020D4
:10408000EBE70000FF030000F0B51C0D671E3F05C5
:10409000DB1BE70A6405640D02D0661CF60A04D037
:1040A000002201231B05803C2403D0252D06002679
:1040B000F6432E661E096E66CE0FF619B446490009
:1040C0004F0D02D07E1CF60A03D000200021403F95
:1040D0003F033E1BB600B444013F7F05C91B49089E
:1040E0002E6F013676089C02950D25437543ED131E
:1040F0007543AD1301356D10F603761B0CB4CC027D
:10410000450D2C43A2B2B3B25A43270C7B43350C66
:104110006F43A4B26C431B1902D3012424043F193A
:104120001C041D0CA4187D4124196D41009A91B204
:10413000ACB26143170C7C432B0C5F4392B25A43E1
:10414000A41802D301221204BF182204230C52180F
:104150007B41019C6C431B19520ED9010A43440157
:10416000A01A81B2B2B2514303145A43360C7343BE
:1041700087B27743D617D21900277E4136049B19A0
:104180001704160C7F185E417316ED18F301002614
:1041900080337541A90F06D16400690AE8055B0AFE
:1041A000184309D22FE00422944480337541A90AB0
:1041B000A8059B0A184326D3404149412404009A8C
:1041C000019B0D005543641B4343E41A95B286B22C
:1041D0007543170C7E43030C5F4392B25A43B618E3
:1041E00002D301221204BF183204330C52197B414E
:1041F00052429C41002C02D400220130514140081F
:10420000CA071043490802B06246D7079210084B0C
:10421000D218084B9A4203D212058918C919F0BD69
:104220000020002A01DC3900F0BD01331905F5E753
:10423000FD030000FE070000002200B5203200F060
:1042400004F8080000BD000000220B150AD410B5C8
:10425000944600F031F81414013400DA0021CB1731
:10426000144C20470020002170476244343A0CD49B
:104270000C2A07DA04009140904052422032D44088
:10428000214310BDD843D94310BD203207D40C467A
:104290009440524220321141D040204310BD0800CA
:1042A000C917203203D452422032104110BD1800E9
:1042B000190010BD6B4200100A0DCC0F531E1B05D8
:1042C000C91A520503D3C943404200D30131520DEC
:1042D00003D0531CDB0A07D0121B00206400611CB2
:1042E00089078912803A1203014BD21A70470000E5
:1042F000FF03000051434343C9188C46110C83B29D
:104300004B4310B4040C614392B280B250436243F9
:104310001C041B0C001910BC59411304120CC018CA
:1043200051416144704700004840414048400023EB
:104330009C46114B5B68184700239C460E4B1B683C
:1043400018470E4A936F9B0804D200239C460A4BE1
:10435000DB681847F0B5146E556E576F166FFFF790
:10436000F4FF064A1466556657671667F0BD0023CA
:104370009C46014B9B6818474C0C0020000000D065
:10438000491A002808D1084670470000C10FC90724
:1043900000D54042002817D0F44603B40B4B1B68ED
:1043A000984706BC81409E384042803107D20B06B8
:1043B00007D04900490AC00510430843604701304F
:1043C000F8E7490A8902F5E770470000480C002029
:1043D00000239C46014B5B6A184700004C0C0020F0
:1043E00070B513231E782A48FFF7FAF80500012E4E
:1043F00011D0012E09DDAB1E1B789B007F2B40DD09
:1044000024488022290000F0AFF82348FFF7E0F8A5
:10441000224B186070BD1F485422290000F0A4F8F8
:104420001F4B1A881F4B9A421CD1A7239B011A8845
:104430001D4B9A4216D11D4B1A881D4B9A4211D121
:104440001C4B1A8894239B019A420BD11A4B1A8851
:104450001A4B9A4206D11A4B1A681A4B9A4201D14A
:10446000152307E01848FDF7B7FF184C094A9900D3
:104470008C5001331F2BF8D9144B064A1362D361B9
:10448000B7E7134B134A14484221FDF70DFFC0460E
:10449000534600004C0C00204C330000480C002018
:1044A000EE290000C40F0000C20D0000962B000092
:1044B000C0B50000182B0000CC2A000010B5000089
:1044C000FC2C000051ED8764C45F0010DD44001037
:1044D00058630010DC6300108C63001007B5604661
:1044E000002800D100BE01880A0A0230DF2AFAD172
:1044F000C9B2820804D3028840880004104300E057
:104500000068024A5050039007BD00004C0C002088
:1045100010B5002804D04018034B984200D810BDB5
:104520000248FDF759FFC04600000420F063001068
:1045300070B5050000F024FB04002900FFF7E8FF38
:10454000200070BD10B500F025FB10BD014804210E
:10455000014B1847C0020020F1350010014B1B68C9
:1045600018470000C0020020014B5B68184700009C
:10457000C002002010B50300080011001B68984716
:1045800010BD0000F8B507000D001600437D002B9C
:1045900002D0002400200CE0036811002800984796
:1045A0002DE03B7D10E03B68154802219847601CD8
:1045B0000134B44214DA002CF3DD2B19013B1B78D3
:1045C0000D3B5A425341DBB22A5D0A2AF0D1002B3F
:1045D000EED1A042E7DA3B68211A28189847E2E7B3
:1045E000B04203DA3B68311A28189847002E06DDDE
:1045F000AD19013D2B780D3B5A4253413B75F8BD37
:104600006064001070B505000368002B16D00C4BD9
:104610001C6805E0290004C92000FFF7B3FF2469E6
:10462000002C09D02368002BF9D0064B1B68002B07
:10463000F0D0A342F3D1EDE700232B6070BDC0465C
:10464000280B0020300B002070B505000C000B6813
:10465000802B05D023685A1C2260E418257170BD98
:104660000800FFF7CFFFF5E710B5002B02DB026073
:10467000436010BD024B034A03483F21FDF714FE7F
:104680009455001064640010B055001010B582B04D
:104690000400FDF7BBF902000B006846FFF7E4FFDA
:1046A000009A019B22606360200002B010BD0000F0
:1046B00070B582B0060014001D00FA22920000239B
:1046C00006980021FFF716FE02000B0012196B413D
:1046D000002B09DB6846FFF7C7FF009A019B326099
:1046E0007360300002B070BD01225242004BF1E70E
:1046F000FFFFFF7F30B585B004000D0002A8FFF773
:10470000C5FF029A039B00952000FFF7D1FF200010
:1047100005B030BD00B583B0FA2189006846FFF7C7
:10472000E9FF009A019B024800F0D6FE03B000BDED
:104730000808002010B5024800F0B6FE10BDC046C3
:1047400008080020F0B5CE46474680B583B0060085
:104750000D0090461C00FFF7DDFF81466B1C05D065
:10476000002C08D0194F1A4B1C6807E0300000F0ED
:1047700027FD0500F4E7174FF5E72469002C17D053
:104780002368002BF9D0144B1B68002B01D0A342E7
:10479000F3D12A0031002000B8474346002BECD06B
:1047A0006B46D91D0A230B7001222000B847E4E7AD
:1047B0004B46002B07D16B1E9D41E8B203B0C0BC35
:1047C000B946B046F0BDFFF7B5FFF4E775450010F8
:1047D000280B002085450010300B002010B5064B3B
:1047E0001C6801E098472469002C03D06368002B03
:1047F000F8D1F8E710BDC046280B002070B50500C1
:1048000000F0DEFC04000023012201002800FFF775
:1048100099FFFFF7E3FF200070BD000070B5A2B064
:1048200004000E00FFF776FF0500002301930A48FD
:104830003300220001A9FEF7B3FE040001A8FFF730
:10484000E1FEFFF7CBFF002D02D1200022B070BDAA
:10485000FFF770FFF9E7C046494600100FB400B5F6
:1048600083B004A901C90191FFF7D8FF03B008BCC8
:1048700004B0184710B5040010220021FFF76EFEA7
:1048800080235B022360F8235B0263608023DB02EA
:10489000A360C0231B03A360200010BD0523CB56DB
:1048A000002B01DB934211D1094B9C4660444342EB
:1048B0005841084B8000C058097901238B40013BC7
:1048C0009340184043425841C0B270470020FCE773
:1048D0000000D0AFA40A002070B50A79202A19D8A8
:1048E000174B9C46604443425841164B8000C458C5
:1048F00001239340013B497949B2002910DB0800AC
:104900002025AA1A914218DC8B401C4201D00120BC
:10491000404270BD0C4B0D4A0D484021FDF7C4FCD0
:104920002020801A002805DB1A0082401442F0D0B3
:104930000138F7E701204042EBE701204042E8E779
:104940000000D0AFA40A00207C64001004650010B1
:10495000A864001070B505000C001600FFF79EFF5C
:10496000002801D0002108E01648FDF735FD9A190E
:104970008B1912339B005A51013123798B4211D983
:10498000227863781B021343A27812041A43E37857
:104990001B0613434A009B5A802292019342E6D39E
:1049A0001A00E5E701229A401300013B064A9446AB
:1049B00065446A4255410549AD006A58B340134306
:1049C0006B5070BDF06400100000D0AFA40A00204E
:1049D000F8B505000E00FCF749F807003100280083
:1049E000FFF77AFF041E09DB020031002800FFF701
:1049F000B1FF3800FCF746F82000F8BD0148FDF78C
:104A0000EBFCC046F0640010F0B5C64600B506AC3D
:104A100025784C006618F60086193700DC373F68A9
:104A2000BC46CC363668B0466418E400C834041975
:104A30000434C026B60134438026B6022660002D19
:104A400001D01F2614E0002612E05401A0256D05B8
:104A500025434C006418E40004192700DC373D604E
:104A6000114D3543D8342560053B05321F242240C3
:104A7000052BEAD89B06520113434C006218D20062
:104A800082181500DC352B60074B3343D832136096
:104A900063462B606418E4000019CC304346036081
:104AA00080BCB846F0BDC04680E0000070B584B060
:104AB00004000D00160002680121A9408A4302602B
:104AC000002B34D0186869004919C90061180A0020
:104AD000C832106058680432106098680432106060
:104AE000DB68DC310B606A005319DB00D033E3185C
:104AF000802149010B438021090619601960164B7A
:104B0000AB40A3602B1D01210800984080239B012E
:104B10002343186028000830814019601F23334068
:104B20005219D200A418D834236004B070BD68466E
:104B3000FFF7A0FE00996B005B19DB00E3181A0079
:104B4000C832116001990432116002990432116077
:104B5000039ADC331A60C6E70101010110B582B087
:104B60000100054C054B00930B2300222000FBF7AE
:104B7000ACFF02B010BDC046840D002024650010BB
:104B800010B5034B0100186800F00EF810BDC046C8
:104B9000E006002010B5034B0100186800F098FBF8
:104BA00010BDC046E0060020F0B54E464546DE4644
:104BB0005746E0B50D000B35060085B0162D27D8F9
:104BC000102900D9DAE000F0D1FA102518230221CB
:104BD000C74FFB181A005C68083A944200D146E1BE
:104BE00003226368A1689343E268CA60916001216F
:104BF000E3185A6830000A435A6000F0B9FA2000FE
:104C0000083005B0F0BCBB46B246A946A046F0BD90
:104C100007239D4300D5B1E0A94200D9AEE000F0E2
:104C2000A5FAFC235B009D4200D29AE1690A00D1FB
:104C3000A8E0042900D94FE138239846A9098844FF
:104C40003931CB00082252429446A94FFB189C44AC
:104C50006346DC68A44514D0032399460B006146E3
:104C60009C4607E0E068002A00DBFAE0814200D1C0
:104C7000FBE004004A46636893435A1B0F2AF1DDA8
:104C800041463A003C690832944200D1D8E0032002
:104C900063688343581B0F2800DD66E13A617A613F
:104CA0000028A4DA7A68904680229200934200D3CA
:104CB000E3E0DA0858090123834040461843804660
:104CC000D300DB199A687860E360A2609C60D460CE
:104CD00001208B10984040455CD8434603420AD1DE
:104CE00003239943434640000431034203D140006B
:104CF00004310342FBD00323B3469C460E00B84662
:104D00000190F00040440100B246CB680BE06446DD
:104D10005A681F00A243DB68541B0F2C00DDF3E030
:104D2000002C00DB0DE19942F1D101239946CA44E0
:104D3000534608319B07E8D1032205E00368083891
:104D4000013E834200D00AE23242F7D14346019A43
:104D50005B68934342465360019A520001929A4223
:104D600016D8002A06D113E004229146019ACA44BB
:104D7000520001921342F7D05646C2E70C2300209E
:104D800033603EE780233F22402190469B0059E755
:104D90005E4647460322BC68636893439946AB422C
:104DA00002D35B1B0F2B4EDC23004B440293514B71
:104DB00008201B6810335B19019300F0F3F94E498A
:104DC00003900B688B46013306D08446019B424218
:104DD000013B6344134001933000019900F0CAF98C
:104DE00003008046013300D1DDE0029B834200D9FD
:104DF000D7E0019A414B944619689A466144039A58
:104E00001960029B0800013A434500D0EAE043469E
:104E1000134200D0E6E0BB68984663464B441A0054
:104E200001231A4343465A60354B1868884200D222
:104E30001960344B1868884200D219604446B4E0C7
:104E40007B68984644E70122290013431143651902
:104E500061603000BD606B6000F08AF920000830AE
:104E6000CFE6A268D0608260C1E6614609E7DC68EF
:104E70000231A34200D104E7B2E65A0A042A00D85C
:104E800088E0142A00D90FE110005B3082465C32C2
:104E9000D200082040428446BA1894446246926880
:104EA0000B308146944500D1E5E00800A2466146FA
:104EB000844602E09268914204D04C465068A04378
:104EC0009842F7D8D368614654469C466346A26030
:104ED000E3609C60D460FBE6142973D9542900D99F
:104EE000EBE06E239846290B88446F31CB00A9E68E
:104EF000D802002074090020D002002044090020BC
:104F00006C09002070090020BA46012051468446F1
:104F10004919054350464560856847466046EB6041
:104F20005E469D6053463961796120430837486089
:104F3000CF6030008F609C5000F01AF95046083066
:104F40005FE6BA4601205E46524451680143516013
:104F5000BA683000D3609A6000F00AF9380008306F
:104F60004FE62B00E908083332E661198846012133
:104F70008C460D434146656039617961CA608A603B
:104F8000624602434A60E050300000F0F1F8200031
:104F9000083036E69A091000393238308246D2009D
:104FA00077E7BC4214D0BC68626803239A43531B62
:104FB000AA4202D30F2B00DD45E7300000F0D8F8FD
:104FC00000201EE65B23984688445C31CB0039E61E
:104FD000644B9A461868019B9C465346604418608F
:104FE000039B5A1E5B461B68013371D043460299EE
:104FF0005B1A51461B180B60072341464046194077
:105000000291184240D00398013384465B1A0199FB
:10501000984441440191634411405B1A1A401100C5
:105020003000934600F0A6F8431C78D04346C01ADF
:1050300003005B44019353461968012059441960E9
:105040004346019ABB6002435A60BC4200D1EBE682
:105050004B460F2B40D907220C3B9343626802401A
:1050600005201A436260E218506090600F2B4BD805
:1050700043465A68D8E65346981001238340404679
:1050800018438046786021E7019B0399434413400D
:10509000CB1A1A4011003000934600F06BF8431C05
:1050A000C4D100239B46C6E7542A18D81A0B100017
:1050B0006F326E308246D200EBE6AA235B00994243
:1050C00018D8DD3B9846E90B88447831CB00B9E528
:1050D0005B46414619608FE7434658606DE7AA205A
:1050E0004000824226D8DA0B1000783277308246B0
:1050F000D200CEE61C4B994226D87C239846A90CB8
:1051000088447D31CB009DE521003000083100F05E
:10511000DFF853461968BB6898465A6884E6019AD6
:10512000029B94464246083B63449B1A019300232A
:105130009B4680E70C4882420CD89A0C10007D32C6
:105140007C308246D200A4E6FE237E227F21904658
:105150009B0077E5FE227E209200824699E6434638
:105160005B68F9E544090020540500007047C0461B
:105170007047C046002370B5064C05000800236048
:10518000FDF772F8431C00D070BD2368002BFBD0E4
:105190002B60F9E72C0B0020014B18687047C046C4
:1051A000E0060020802310B55B01082801D118001B
:1051B00010BDFFF7F1FF16230360173BF7E7C0466A
:1051C00010B583070AD00300032102E001330B422C
:1051D00005D01A78002AF9D1181A10BD03001968F1
:1051E0000C4A0D4C8A188A4322420FD15968094A49
:1051F00004338A188A43224208D15968054A043385
:105200008A188A432242F1D000E001331A78002A3A
:10521000FBD1E1E7FFFEFEFE80808080F0B5C64650
:10522000060000B508200D00FFF7BCFF04003000A9
:10523000FFF79CFF234B210098469B685F68032380
:105240009F4338001138401B0019FEF715FA451E20
:105250006543AC4208DC00213000FFF78BFF43467A
:105260009B68DB19984206D03000FFF781FF0020D1
:1052700080BCB846F0BD30006942FFF77BFF0130CB
:105280000ED0012243467F1B9B6817430E4A5F6086
:10529000136830005B1B1360FFF76AFF0120E7E72C
:1052A00000213000FFF766FF43469A68831A0F2BF0
:1052B000DADD064C04492468001B086001210B4319
:1052C0005360D1E7D802002044090020D00200201A
:1052D000F8B5CE46474605000C0080B5002957D0EA
:1052E000FFF744FF012321009C46083948686246C5
:1052F000030003249343CF187A68654EA243B46831
:10530000BC4200D170E0BC18A14664467A600442F9
:1053100021D10868091A1B188868804648464068E9
:105320002040340008348146A04551D04046CC6826
:10533000C460A0604846002811D19B185548BA683F
:10534000824200D17FE0F868D060826001221A4377
:105350004A60CB5007E0484640682042EDD06246A4
:105360001A434A603B6080229200934214D2DA08CA
:10537000580901238340706803437360D3009B196D
:105380009A68CB608A609960D1602800FFF7F0FED0
:10539000C0BCB946B046F8BD5C0A042C3DD89C0997
:1053A000200039343830E40034192268083C0327DF
:1053B000944203D140E09268944203D05068B843CD
:1053C0009842F8D8D468CC608A60A160D160DCE7EC
:1053D000002858D1B868D218FB68C360986063464B
:1053E00013434B608A50D0E79A186346034206D1B4
:1053F0000B68C91A8868D218CB68C360986001230B
:1054000013434B60244BB1601B689342BDD8234BC0
:1054100028001968FFF702FFB7E7142C07D9542CAE
:105420001AD81C0B20006F346E30E400BCE720005B
:105430005C345B30E400B7E7012380108340706880
:1054400003437360BFE7D1609160CA608A60012244
:105450001A434A60CB5098E7AA225200944205D8DA
:10546000DC0B200078347730E4009DE70C4A94424E
:1054700005D89C0C20007D347C30E40094E7FE24A9
:105480007E20A40090E762461A434A603B607CE7B6
:10549000D8020020E0020020D4020020740900207D
:1054A00054050000F8B5C04601B40248844601BC6A
:1054B000604700BFC901002001B40248844601BC16
:1054C000604700BF1502002001B40248844601BCB9
:1054D000604700BF1502002001B40248844601BCA9
:0854E000604700BF95010020A8
:1054E80053797374656D20636C6F636B206F6620EE
:1054F8002575206B487A2063616E6E6F7420626533
:105508002065786163746C79206163686965766584
:1055180064000000636861696E5F746F203C3D2021
:105528004E554D5F444D415F4348414E4E454C53A7
:10553800000000002F686F6D652F737069646572D5
:105548005F7069672F7372632F632F7069636F2FA2
:105558007069636F2D73646B2F7372632F7270326F
:105568005F636F6D6D6F6E2F6861726477617265CE
:105578005F646D612F696E636C7564652F68617215
:1055880064776172652F646D612E680075735F734F
:10559800696E63655F626F6F74203C3D20494E54AD
:1055A80036345F4D415800002F686F6D652F73705A
:1055B800696465725F7069672F7372632F632F70F8
:1055C80069636F2F7069636F2D73646B2F737263D8
:1055D8002F636F6D6D6F6E2F7069636F5F6261739C
:1055E800652F696E636C7564652F7069636F2F74BE
:1055F800797065732E6800007570646174655F75F5
:10560800735F73696E63655F626F6F74000000009B
:105618006368616E6E656C5F636F6E6669675F7302
:1056280065745F636861696E5F746F000000205085
:10563800000000001200000011000000150000002A
:105648001300000014000000100000004001E001F9
:105658006056001002FF0000016042B00114010111
:105668000A1102023A550200360005002A0000011C
:105678004005002B000001E001021301022900008F
:1056880030783163203D3D20282A696E7374293EA5
:105698003E313175000000002F686F6D652F737003
:1056A800696465725F7069672F7372632F632F7007
:1056B80069636F2F7069636F2D73646B2F737263E7
:1056C8002F7270325F636F6D6D6F6E2F68617264D9
:1056D800776172655F6972712F6972712E6300005C
:1056E80064656C7461203E3D202D323034382026AC
:1056F800262064656C7461203C3D203230343620AD
:10570800262620212864656C746120262031290012
:10571800212864656C7461203E3E20313175290072
:1057280063757272656E74203D3D205F5F756E68AB
:10573800616E646C65645F757365725F6972712010
:105748007C7C2063757272656E74203D3D206861B3
:105758006E646C6572000000216578636570746919
:105768006F6E207C7C20657863657074696F6E202D
:105778003D3D206E756D202B20565441424C455FAF
:1057880046495253545F49525100000066616C7398
:105798006500000069735F7368617265645F6972B0
:1057A800715F7261775F68616E646C657228736C93
:1057B8006F745F68616E646C6572290065786365F3
:1057C8007074696F6E000000666F756E640000008B
:1057D8006972715F6164645F7461696C5F746F5F43
:1057E800667265655F6C697374000000696E736545
:1057F80072745F6272616E63685F616E645F6C6928
:105808006E6B00006972715F72656D6F76655F68B7
:10581800616E646C657200006D616B655F627261D8
:105828006E6368007265736F6C76655F6272616E35
:10583800636800006972715F7365745F6578636C93
:1058480075736976655F68616E646C6572000000E7
:10585800746F74616C0000002F686F6D652F737032
:10586800696465725F7069672F7372632F632F7045
:1058780069636F2F7069636F2D73646B2F73726325
:105888002F636F6D6D6F6E2F7069636F5F73796EC5
:10589800632F6D757465782E630000006D74782D24
:1058A8003E636F72652E7370696E5F6C6F636B0019
:1058B8006C6F636B5F69735F6F776E65725F696446
:1058C8005F76616C6964286D74782D3E6F776E65BC
:1058D800722900006D74782D3E656E7465725F6381
:1058E8006F756E74000000006D757465785F65787B
:1058F800697400006D757465785F656E7465725FB4
:10590800626C6F636B5F756E74696C0069642026E6
:1059180026206964203C3D20706F6F6C2D3E6865C1
:1059280061702D3E6D61785F6E6F64657300000075
:105938002F686F6D652F7370696465725F70696732
:105948002F7372632F632F7069636F2F7069636F92
:105958002D73646B2F7372632F636F6D6D6F6E2F72
:105968007069636F5F74696D652F74696D652E6307
:10597800000000006964202626206964203C3D2040
:10598800686561702D3E6D61785F6E6F6465730048
:105998002F686F6D652F7370696465725F706967D2
:1059A8002F7372632F632F7069636F2F7069636F32
:1059B8002D73646B2F7372632F636F6D6D6F6E2F12
:1059C8007069636F5F7574696C2F696E636C756459
:1059D800652F7069636F2F7574696C2F70686561C6
:1059E800702E6800706172656E745F6964000000F3
:1059F8006368696C645F69640000000070617265C7
:105A08006E745F696420213D206368696C645F6916
:105A18006400000069640000696420262620217063
:105A2800685F636F6E7461696E735F6E6F6465281B
:105A3800686561702C20696429000000216865612F
:105A4800702D3E667265655F7461696C5F6964009C
:105A58002170685F636F6E7461696E735F6E6F64E7
:105A68006528706F6F6C2D3E686561702C207265BB
:105A78007573655F6964290072656D6F7665645F2B
:105A88006964203D3D206E6578745F69640000009C
:105A980063616C6C6261636B00000000706F6F6C17
:105AA8002D3E616C61726D5F696E5F70726F6772B7
:105AB800657373203D3D206D616B655F7075626C29
:105AC80069635F69642869645F686967682C206E28
:105AD8006578745F6964290064656661756C745FD4
:105AE800616C61726D5F706F6F6C5F696E6974690C
:105AF800616C697A6564282900000000616C617234
:105B08006D5F696420213D20706F6F6C2D3E616C64
:105B180061726D5F696E5F70726F67726573730033
:105B280072630000417474656D7074656420746FED
:105B380020736C65657020696E73696465206F6693
:105B480020616E20657863657074696F6E20686186
:105B58006E646C65723B2075736520627573795F3E
:105B68007761697420696620796F75206D75737423
:105B780000000000616C61726D5F706F6F6C5F6335
:105B8800616E63656C5F616C61726D00616C6172FE
:105B98006D5F706F6F6C5F6765745F646566617574
:105BA8006C7400006765745F656E7472795F696410
:105BB8005F6869676800000070685F667265655FA6
:105BC8006E6F64650000000070685F6164645F6305
:105BD80068696C645F6E6F646500000070685F6977
:105BE8006E736572745F6E6F6465000070685F67DE
:105BF80065745F6E6F6465006164645F616C617297
:105C08006D5F756E6465725F6C6F636B000000009A
:105C18007570646174655F75735F73696E63655FE2
:105C2800626F6F7400000000616C61726D5F706F6D
:105C38006F6C5F616C61726D5F63616C6C626163F4
:105C48006B0000006765745F656E74727900000010
:105C5800486172647761726520616C61726D20259C
:105C68006420616C726561647920636C61696D653B
:105C78006400000074696D65725F68772D3E696E17
:105C880074732026203175203C3C20616C61726D54
:105C98005F6E756D000000002F686F6D652F737063
:105CA800696465725F7069672F7372632F632F7001
:105CB80069636F2F7069636F2D73646B2F737263E1
:105CC8002F7270325F636F6D6D6F6E2F68617264D3
:105CD800776172655F74696D65722F74696D65723D
:105CE8002E63000068617264776172655F616C6140
:105CF800726D5F7365745F7461726765740000002C
:105D0800726F6F745F6964002F686F6D652F7370B1
:105D1800696465725F7069672F7372632F632F7090
:105D280069636F2F7069636F2D73646B2F73726370
:105D38002F636F6D6D6F6E2F7069636F5F75746918
:105D48006C2F70686561702E630000002170685FB9
:105D58006765745F6E6F646528686561702C207272
:105D68006F6F745F6964292D3E7369626C696E6731
:105D7800000000002170685F6765745F6E6F64657E
:105D880028686561702C20726F6F745F6964292DB3
:105D98003E706172656E74006E65775F7375625FE1
:105DA8007472656520213D20686561702D3E726FB3
:105DB8006F745F696400000070685F72656D6F766C
:105DC800655F616E645F667265655F6E6F646500CE
:105DD80070685F72656D6F76655F616E795F686523
:105DE8006164000070685F6164645F6368696C6423
:105DF8005F6E6F646500000070685F6765745F6E52
:105E08006F6465007372635F66726571203E3D2042
:105E180066726571000000002F686F6D652F7370E2
:105E2800696465725F7069672F7372632F632F707F
:105E380069636F2F7069636F2D73646B2F7372635F
:105E48002F7270325F636F6D6D6F6E2F6861726451
:105E5800776172655F636C6F636B732F636C6F63DD
:105E68006B732E6300000000636C6F636B5F636F7E
:105E78006E6669677572650076636F5F66726571D5
:105E8800203E3D20285049434F5F504C4C5F5643BD
:105E98004F5F4D494E5F465245515F4D485A202A43
:105EA800204D485A292026262076636F5F66726542
:105EB80071203C3D20285049434F5F504C4C5F5661
:105EC800434F5F4D41585F465245515F4D485A20F8
:105ED8002A204D485A2900002F686F6D652F73706E
:105EE800696465725F7069672F7372632F632F70BF
:105EF80069636F2F7069636F2D73646B2F7372639F
:105F08002F7270325F636F6D6D6F6E2F6861726490
:105F1800776172655F706C6C2F706C6C2E6300001B
:105F28006662646976203E3D20313620262620664A
:105F380062646976203C3D203332300028706F73EC
:105F4800745F64697631203E3D203120262620701A
:105F58006F73745F64697631203C3D2037292026B1
:105F6800262028706F73745F64697632203E3D2066
:105F78003120262620706F73745F64697632203C66
:105F88003D203729000000007265665F6D687A2041
:105F98003C3D202876636F5F66726571202F203143
:105FA80036290000706C6C5F696E6974000000002F
:105FB8002C2066756E6374696F6E3A2000000000CD
:105FC800617373657274696F6E202225732220666F
:105FD80061696C65643A2066696C652022257322C4
:105FE8002C206C696E65202564257325730A0000D2
:105FF80031203D3D202875696E747074725F742974
:106008006C2D3E7370696E5F6C6F636B00000000EF
:106018002F686F6D652F7370696465725F7069674B
:106028002F7372632F632F7069636F2F7069636FAB
:106038002D73646B2F7372632F7270325F636F6D91
:106048006D6F6E2F7069636F5F72756E74696D65C1
:106058002F72756E74696D652E6300000A2A2A2AEC
:106068002050414E4943202A2A2A0A000A000000EB
:1060780072756E74696D655F696E69740000000001
:10608800666E692B00000000666E69006E616E0026
:10609800666E692D00000000A62F0010BE2F0010AC
:1060A800BE2F0010B22F0010BE2F0010BE2F001000
:1060B800BE2F0010BE2F0010BE2F0010BE2F0010E4
:1060C800BE2F00109A2F0010BE2F00108E2F001028
:1060D800BE2F0010BE2F0010822F00108E3000102F
:1060E800B4300010D6300010B43000106E300010FC
:1060F800B4300010B4300010B4300010B4300010C8
:10610800B4300010B4300010B4300010AA300010C1
:10611800B4300010B4300010B4300010B4300010A7
:10612800B4300010E2300010463500105C35001025
:106138005C3500105C3500105C3500105C350010D3
:106148005C3500105C3500105C3500105C350010C3
:106158005C3500105C3500105C3500105C350010B3
:106168005C3500105C3500105C3500105C350010A3
:106178005C3500105C3500105C3500105C35001093
:106188005C3500105C3500105C3500105C35001083
:106198005C3500105C3500105C3500105C35001073
:1061A8005C3500105C350010883300104A3300104D
:1061B800883300105C3500105C3500105C35001029
:1061C8005C3500105C3500105C3500105C35001043
:1061D8005C3500105C3500105C3500105C35001033
:1061E8005C3500105C3500105C3500105C35001023
:1061F8005C3500102E3100105C3500105C35001045
:106208005C3500105C3500105C3500105C35001002
:106218005C3500105C3500105C3500102E31001024
:10622800D63300102E310010883300104A33001086
:106238008833001000000000000000000000F03F5C
:106248000000000000002440000000000000594049
:106258000000000000408F40000000000088C3409C
:1062680000000000006AF8400000000080842E4111
:1062780000000000D01263410000000084D797415D
:106288000000000065CDCD412A282875696E743854
:106298005F74202A29282828766F6964202A2972A1
:1062A8006F6D5F646174615F6C6F6F6B757028727E
:1062B8006F6D5F7461626C655F636F6465282753F7
:1062C800272C202746272929292D322929202A2029
:1062D80034203E3D2053465F5441424C455F563280
:1062E8005F53495A450000002F686F6D652F737022
:1062F800696465725F7069672F7372632F632F70AB
:1063080069636F2F7069636F2D73646B2F7372638A
:106318002F7270325F636F6D6D6F6E2F7069636F70
:106328005F646F75626C652F646F75626C655F6919
:106338006E69745F726F6D2E630000005F5F616548
:106348006162695F646F75626C655F696E6974002C
:106358002A282875696E74385F74202A2928726F74
:106368006D5F7461626C652D322929202A203420E2
:106378003E3D2053465F5441424C455F56325F5381
:10638800495A45002F686F6D652F7370696465728F
:106398005F7069672F7372632F632F7069636F2F44
:1063A8007069636F2D73646B2F7372632F72703211
:1063B8005F636F6D6D6F6E2F7069636F5F666C6F73
:1063C80061742F666C6F61745F696E69745F726F58
:1063D8006D2E63005F5F61656162695F666C6F6106
:1063E800745F696E697400004F7574206F66206D64
:1063F800656D6F7279000000446562756700000082
:10640800626F6F74325F7732357130383000000058
:10641800312E352E300000007069636F00000000D7
:10642800636C6163657200004D61792032312032FE
:106438003032330006005250D3F075420064001029
:1064480006005250E182887F08640010060052500E
:10645800BBFF3CB6206400100D0A00007570646133
:1064680074655F75735F73696E63655F626F6F7480
:106478000000000070726F6772616D2D3E6C656E72
:10648800677468203C3D2050494F5F494E53545231
:10649800554354494F4E5F434F554E54000000003A
:1064A8002F686F6D652F7370696465725F706967B7
:1064B8002F7372632F632F7069636F2F7069636F17
:1064C8002D73646B2F7372632F7270325F636F6DFD
:1064D8006D6F6E2F68617264776172655F70696F46
:1064E8002F70696F2E6300004E6F2070726F677295
:1064F800616D207370616365000000005F70696FF3
:106508005F66696E645F6F66667365745F666F72F7
:106518005F70726F6772616D000000004E6F2044FB
:106528004D41206368616E6E656C732061726520F1
:0C653800617661696C61626C65000000B6
:106544003C64001048640010880200105464001079
:0C65540094020010A0020010AC02001025
:1065600003000068EFF3108C72B60268002AFCD0BA
:10657000BFF35F8F04229A56002A0BDB002910D04C
:106580000A6000201B68BFF35F8F00221A608CF343
:1065900010887047D0221206127852B21A71012068
:1065A000F0E70020EEE70000F8B5CE46474680B59C
:1065B0000400170098460368002B20D0D0231B0648
:1065C0001B785BB299462668EFF3108C72B635687B
:1065D000002DFCD0BFF35F8F04256557002D14DB21
:1065E0002368BFF35F8F00221A608CF31088380095
:1065F000414600F069F80028E5D000200FE00A4B82
:106600000A4A0B48852100F057F84B46237123684E
:10661000BFF35F8F00221A608CF310880120C0BC8A
:10662000B946B046F8BDC046A4580010FC5800104A
:106630006058001070B582B0060015001C0001A95A
:10664000FFF78EFF002807D1019B5BB2D022120614
:10665000127852B2934201D102B070BD2A002300D9
:106660003000FFF7A1FFF7E710B50268EFF31081E4
:1066700072B61368002BFCD0BFF35F8F0423C356A0
:10668000002B0ADBFF2303710368BFF35F8F002237
:106690001A6081F3108840BF10BD034B034A0448C1
:1066A000B42100F009F8C046B8580010F0580010A6
:1066B000605800107047C04601B40248844601BCCF
:1066C000604700BFA922001001B40248844601BC03
:1066D000604700BF251900101000000000000000F6
:1066E00000000100000000000000000000000200A7
:1066F0000000000000000000000003000000000097
:10670000000000000000FF000000000001B5486824
:1067100001318E460047704609380149884701BD5E
:106720006D0E00109C0200200000000028080020D0
:10673000E40A00200000000000000000F40A00202D
:106740000000000000000000100000000000000039
:10675000503300004C33000054330000523300002B
:106760004D5300004D4300005334000043340000FB
:10677000FFFFFFFF0000020000000000000000001B
:10678000D8020020D8020020E0020020E002002011
:10679000E8020020E8020020F0020020F0020020C1
:1067A000F8020020F802002000030020000300206F
:1067B000080300200803002010030020100300201D
:1067C00018030020180300202003002020030020CD
:1067D000280300202803002030030020300300207D
:1067E000380300203803002040030020400300202D
:1067F00048030020480300205003002050030020DD
:10680000580300205803002060030020600300208C
:10681000680300206803002070030020700300203C
:1068200078030020780300208003002080030020EC
:10683000880300208803002090030020900300209C
:106840009803002098030020A0030020A00300204C
:10685000A8030020A8030020B0030020B0030020FC
:10686000B8030020B8030020C0030020C0030020AC
:10687000C8030020C8030020D0030020D00300205C
:10688000D8030020D8030020E0030020E00300200C
:10689000E8030020E8030020F0030020F0030020BC
:1068A000F8030020F803002000040020000400206A
:1068B0000804002008040020100400201004002018
:1068C00018040020180400202004002020040020C8
:1068D0002804002028040020300400203004002078
:1068E0003804002038040020400400204004002028
:1068F00048040020480400205004002050040020D8
:106900005804002058040020600400206004002087
:106910006804002068040020700400207004002037
:1069200078040020780400208004002080040020E7
:106930008804002088040020900400209004002097
:106940009804002098040020A0040020A004002047
:10695000A8040020A8040020B0040020B0040020F7
:10696000B8040020B8040020C0040020C0040020A7
:10697000C8040020C8040020D0040020D004002057
:10698000D8040020D8040020E0040020E004002007
:10699000E8040020E8040020F0040020F0040020B7
:1069A000F8040020F8040020000500200005002065
:1069B0000805002008050020100500201005002013
:1069C00018050020180500202005002020050020C3
:1069D0002805002028050020300500203005002073
:1069E0003805002038050020400500204005002023
:1069F00048050020480500205005002050050020D3
:106A00005805002058050020600500206005002082
:106A10006805002068050020700500207005002032
:106A200078050020780500208005002080050020E2
:106A30008805002088050020900500209005002092
:106A40009805002098050020A0050020A005002042
:106A5000A8050020A8050020B0050020B0050020F2
:106A6000B8050020B8050020C0050020C0050020A2
:106A7000C8050020C8050020D0050020D005002052
:106A8000D8050020D8050020E0050020E005002002
:106A9000E8050020E8050020F0050020F0050020B2
:106AA000F8050020F8050020000600200006002060
:106AB000080600200806002010060020100600200E
:106AC00018060020180600202006002020060020BE
:106AD000280600202806002030060020300600206E
:106AE000380600203806002040060020400600201E
:106AF00048060020480600205006002050060020CE
:106B0000580600205806002060060020600600207D
:106B1000680600206806002070060020700600202D
:106B200078060020780600208006002080060020DD
:106B3000880600208806002090060020900600208D
:106B40009806002098060020A0060020A00600203D
:106B5000A8060020A8060020B0060020B0060020ED
:106B6000B8060020B8060020C0060020C00600209D
:106B7000C8060020C8060020D0060020D00600204D
:106B8000E806002000000000000000007809002056
:106B9000DC090020400A0020000000000000000086
:106BA00000000000000000000000000000000000E5
:106BB00000000000000000000000000000000000D5
:106BC00000000000000000000000000000000000C5
:106BD00000000000000000000000000000000000B5
:106BE00000000000000000000000000000000000A5
:106BF0000000000000000000000000000000000095
:106C00000000000000000000000000000000000084
:106C10000000000000000000000000000000000074
:106C200001000000000000000E33CDAB34126DE611
:106C3000ECDE05000B00000000000000000000007A
:106C40000000000000000000000000000000000044
:106C50000000000000000000000000000000000034
:106C60000000000000000000000000000000000024
:106C70000000000000000000000000000000000014
:106C80000000000000000000000000000000000004
:106C900000000000000000000000000000000000F4
:106CA00000000000000000000000000000000000E4
:106CB0004D450010C1350010C13C0010E1430010EB
:046CC000310300108C
:04000005100001E9FD
:00000001FF
